:100000000C94270C0C941A2A0C94F3290C944F0C82
:100010000C944F0C0C944F0C0C94412A0C944F0CE4
:100020000C944F0C0C94772B0C944F0C0C944F0C9D
:100030000C944F0C0C944F0C0C944F0C0C944F0CD4
:100040000C94A9290C944F0C0C944F0C0C944F0C4D
:100050000C944F0C0C944F0C0C944F0C0C944F0CB4
:100060000C94582A0C944F0C000000000000000073
:10007000000F200000200000001100000020000000
:100080000010000000200000001022CE2C21800073
:100090000010233132224000000C222121242000B4
:1000A0000002222121242000000122212127E0003A
:1000B000000122212124000000012221212400002E
:1000C0000011222132222000001E22212C11C0000A
:1000D0000000000020000000000000000000000000
:1000E0000000000000000000000003C0000000004D
:1000F0000000022000000000000002128600000044
:10010000000002130900000000000212108000002D
:100110000000021210800000000002121080000097
:10012000000003E2108000000000020210800000C6
:10013000000002021080000000000202090000001E
:1001400000000202060000001E0000002000000067
:10015000118000002002000010800000200200003A
:1001600010860D2121E78C281089132121121230CD
:100170001190A121201221201E10A1212012212046
:10018000121FA12121F22120111021212212212050
:1001900011102121221221201088932322321220B3
:1001A00010C70D1D11D18C200000010000000000BF
:1001B000000002000000000000000000000000003D
:1001C00000010200010000000001860001000000A3
:1001D000000186000100000000014A0C0D0C000027
:1001E00000014A121312000000014A2121210000DF
:1001F00000012A212121000000013221213F0000BD
:100200000001122121200000000102212120000014
:1002100000010212131100000001020C0D0E00007B
:1002200000000000000000000000000000000000CE
:100230000048000008000000F248201008004200BA
:10024000804821100800420082481323899C4258AC
:100250008248132049224264824812A04A22424224
:10026000F24814A3CC3E4242824814A44A2042429F
:10027000824814A44A20424282480844C920426469
:1002800082240843499E3C580000000000000040C2
:10029000000000000000004000000000000000001E
:1002A00000000000000000663E0000000001E08841
:1002B0002100000000021088210C2211C50409FE53
:1002C00021122312260408882121132424040888DB
:1002D000232112A4240408883C2114A7E4040888DC
:1002E000202114A404040888202114A404040888EC
:1002F00020120CC224021088200C0841E401E0887E
:1003000000000000000000000000000000000000ED
:1003100000000000000000CC1E0000000000E11002
:100320002000000000011110201CA38397020BFC89
:100330002020C44458820910104088485082091077
:100340000C4088485082091002408FCFD08209109B
:1003500002408808108209100240880810820910A3
:1003600002208444508111103C1C83C3D080E110D2
:10037000000000000000000000000000000000007D
:1003800000000000004000007C0020001E40000033
:100390004200200020400000421E79E04041C78A10
:1003A000411121104042244C41012010404420487A
:1003B0004101201040442048411F21F04047E7C838
:1003C000412122104044084842212210404408485C
:1003D00042232230204228C87C1D19D01E21E74824
:1003E000000000000000000000000000000000000D
:1003F00078000080200000004400000000000000A1
:1004000044059896259912CC4406649926651332C2
:100410004404449124451222440444912445122268
:1004200078E4449124451222400444912445122248
:100430004004449124451222400444912445322230
:10044000400444912444D222000000000000000037
:10045000000000000000000000000000000000009C
:10046000700402001C00000048040200200000008C
:1004700048EEE73020EA631C49141248210C94929C
:100480004914124811089492491412480908949288
:100490007114F2780508F79251151240050884127C
:1004A00049151240050884124915324805089492EE
:1004B0004CE2D13838E873920000000000000000E0
:1004C0000000000000000000000080040000400068
:1004D00080808004000E400288808004001040026A
:1004E00048989305911070E75504A486511049125D
:1004F0005504A484490849125504C4844A04491285
:10050000551CC7844A0249125524C4044A024912A0
:100510005524A4044A024912222C9486440249120A
:1005200022149385841C48E10000000004000000B0
:1005300000000000040000000000000000000000B7
:100540000000021004800000000002100080000083
:1005500000000212C5C00000000002132480000049
:10056000000002122480000000000212248000001B
:10057000000002122480000000000212248000000B
:100580000000021224800000000001E2244000006C
:10059000000000000000000000000000000000005B
:1005A000000000000000000000000000000000004B
:1005B00000000000000003007C00010000100400A7
:1005C0004200000000100400420C850E3012CE18CC
:1005D00041128510481324244122492088122442C4
:1005E0004122492088122442413E4920F8122442E7
:1005F0004120492080122442422029208012244296
:1006000042123110481224247C0E110E3812241884
:1006100000000000000000000000000000000000DA
:100620000000000000000000FF80FF80C180C1804A
:10063000C180C180C180C180C180C180C180C180B2
:10064000C180C180C180C180C180C180C180C180A2
:10065000C180FF80FF80000000000000000000005B
:1006600000000000000000000C001C003C007C00AA
:100670000C000C000C000C000C000C000C000C001A
:100680000C000C000C000C000C000C000C000C000A
:100690000C007F807F800000000000000000000050
:1006A0000000000000000000FF80FF80018001804A
:1006B0000180018001800180018001800180FF8034
:1006C000FF80C000C000C000C000C000C000C0006B
:1006D000C000FF80FF80000000000000000000005C
:1006E0000000000000000000FF80FF80018001800A
:1006F0000180018001800180018001800180FF80F4
:10070000FF800180018001800180018001800180E3
:100710000180FF80FF80000000000000000000005A
:100720000000000000000000C180C180C180C180C5
:10073000C180C180C180C180C180C180C180FF8073
:10074000FF800180018001800180018001800180A3
:100750000180018001800000000000000000000016
:100760000000000000000000FF80FF80C000C0000B
:10077000C000C000C000C000C000C000C000FF80BA
:10078000FF80018001800180018001800180018063
:100790000180FF80FF8000000000000000000000DA
:1007A0000000000000000000FF80FF80C180C0004A
:1007B000C000C000C000C000C000C000C000FF807A
:1007C000FF80C180C180C180C180C180C180C180E3
:1007D000C180FF80FF8000000000000000000000DA
:1007E0000000000000000000FF80FF800180018009
:1007F000018003000300060006000C000C00180036
:100800001800180018001800180018001800180028
:100810001800180018000000000000000000000090
:100820000000000000000000FF80FF80C180C18048
:10083000C180C180C180C180C180C180FF80FF8034
:10084000FF80C180C180C180C180C180C180C18062
:10085000C180FF80FF800000000000000000000059
:100860000000000000000000FF80FF80C180C18008
:10087000C180C180C180C180C180C180FF80FF80F4
:100880000180018001800180018001800180018060
:100890000180FF80FF8000000000000000000000D9
:1008A0000000000000000000000000000000000048
:1008B0000000000000000000000000000000000038
:1008C0000000000000000000000000000000000028
:1008D0000000000000000000000000000000000018
:1008E0000000000000000000000000000000000008
:1008F00000000000000000000000000000000000F8
:1009000000000000000000000000000000000000E7
:1009100000000000000000000000000000000000D7
:1009200000000000000000000000000000000000C7
:1009300000000000000000000000000000000000B7
:1009400000000000000000000000000000000000A7
:100950000000000000000000000000000000000097
:100960000000000000000000000000000000000087
:100970000000000000000000000000000000000077
:100980000000000000000000000000000000000067
:100990000000000000000000000000000000000057
:1009A0000000000000000000000000000000000047
:1009B0000000000000000000000000000000000037
:1009C0000000000000000000000000000000000027
:1009D0000000000000000000000000000000000017
:1009E0000000000000000000000000000000000007
:1009F0003080000000008400110000000000C400EE
:100A0000111870000000A4700A2480000000A4885F
:100A10000A4480000000A4880444800000009488F8
:100A2000047C60000000948804401000000094885A
:100A30000440100000008C880424100000008C8802
:100A4000041CE000000084700000000000000000B2
:100A50000000000000000000000000000000000096
:100A60000000000000000000000000000000000086
:100A7000000001E00800000000000110000000007C
:100A800000000111C8000000000001120800000071
:100A90000000011208000000000001120800000020
:100AA000000001E188000000000001004800000093
:100AB00000000100480000000000010048000000A4
:100AC000000001038800000000000000000000009A
:100AD0000000000000000000000000000000000016
:100AE0000000000000000000000000000000000006
:100AF000000001E000000000000001100000000004
:100B000000000111C50000000000011026000000D7
:100B10000000011024000000000001E0240000009B
:100B200000000111E4000000000001122400000098
:100B30000000011224000000000001126400000007
:100B4000000001E1A400000000000000000000001F
:100B50000000000000000000000000000000000095
:100B60000000000000000000000000000000000085
:100B700000000038000000000000004400000000F9
:100B800000000082580000000000008264000000A5
:100B900000000082440000000000008244000000C9
:100BA00000000082440000000000008244000000B9
:100BB00000000082440000000000004444000000E7
:100BC00000000038440000000000000000000000A9
:100BD0000000000000000000000000000000000015
:100BE000000000000000000000000000660000009F
:100BF0000000003888000000000000448800000069
:100C000000000083FC00000000000082880000005B
:100C100000000082880000000000008288000000C0
:100C200000000082880000000000008288000000B0
:100C300000000082880000000000004488000000DE
:100C400000000038880000000000000000000000E4
:100C50000000000000000000000000000000000094
:100C60000000000000000000000000200000000064
:100C70000000072000000000000008200000000025
:100C8000000010218714000000001022409800008E
:100C9000000010244090000000001024409000004C
:100CA00000001027C79000000000102408900000EA
:100CB0000000102408900000000008224990000065
:100CC00000000711C69000000000000000000000B6
:100CD0000000000000000000000000000000000014
:100CE0000000000000000000000000000000000004
:100CF00000003C0000000000000022000000400056
:100D00000000211C583040000000212264484000AF
:100D10000000212244884000000021224488400035
:100D20000000212244F840000000212244804000BD
:100D3000000021224480400000002222444800009C
:100D400000003C1C4438400000000000000000008F
:100D50000000000000000000000000000000000093
:100D60000000000000000000000000000000000083
:100D700000000413E3C00000000002220400000091
:100D800000000222040000000000014204000000F4
:100D9000000001420200000000000083C18000004A
:100DA00000000082004000000000008200400000BF
:100DB00000000082004000000000008200400000AF
:100DC00000000083E7800000000000000000000039
:100DD0000000000000000000000000000000000013
:100DE0000000000000000000000000000000000003
:100DF000000000C21C000000000000C22200000031
:100E0000000000A241000000000000A2410000001C
:100E1000000000924100000000000092410000002C
:100E20000000008A410000000000008A410000002C
:100E30000000008641000000000000862200000043
:100E4000000000821C000000000000000000000004
:100E50000000000000000000000000000000000092
:100E6000000000000000FFF8FFF8FFF8E038E0386D
:100E7000E038E038E038E038E038E038E038E038B2
:100E8000E038E038E038E038E038E038E038E038A2
:100E9000E038FFF8FFF8FFF8000000000000000055
:100EA00000000000000007000F001F001F007F006F
:100EB000770067000700070007000700070007002A
:100EC00007000700070007000700070007000700EA
:100ED0000700FFF0FFF0FFF000000000000000003E
:100EE000000000000000FFF0FFF0FFF00070007055
:100EF000007000700070007000700070FFF0FFF074
:100F0000FFF0E000E000E000E000E000E000E000D2
:100F1000E000FFF0FFF0FFF0000000000000000024
:100F2000000000000000FFF0FFF0FFF00070007014
:100F3000007000700070007000700070FFF0FFF033
:100F4000FFF00070007000700070007000700070A2
:100F50000070FFF0FFF0FFF0000000000000000054
:100F6000000000000000E070E070E070E070E070F1
:100F7000E070E070E070E070E070E070FFF0FFF0B3
:100F8000FFF0007000700070007000700070007062
:100F90000070007000700070000000000000000091
:100FA000000000000000FFF0FFF0FFF0E000E000B4
:100FB000E000E000E000E000E000E000FFF0FFF013
:100FC000FFF0007000700070007000700070007022
:100FD0000070FFF0FFF0FFF00000000000000000D4
:100FE000000000000000FFF0FFF0FFF0E070E07094
:100FF000E070E000E000E000E000E000FFF0FFF063
:10100000FFF0E070E070E070E070E070E070E070C1
:10101000E070FFF0FFF0FFF00000000000000000B3
:10102000000000000000FFF0FFF0FFF0007000F093
:1010300000E00380038007000F001E001C001C005E
:101040001C001C001C001C001C001C001C001C00C0
:101050001C001C001C001C00000000000000000020
:10106000000000000000FFF0FFF0FFF0E070E07013
:10107000E070E070E070E070E070E070FFF0FFF0B2
:10108000FFF0E070E070E070E070E070E070E07041
:10109000E070FFF0FFF0FFF0000000000000000033
:1010A000000000000000FFF0FFF0FFF0E070E070D3
:1010B000E070E070E070E070E070E070FFF0FFF072
:1010C000FFF0007000700070007000700070007021
:1010D0000070FFF0FFF0FFF00000000000000000D3
:1010E0000000000000000000000000000000000000
:1010F00000000000000000000000000000000000F0
:101100000000000000000000000000000000E330CC
:10111000949E90929090E3909490949093D0E0005D
:1011200000000000240254774452275215525552B1
:101130002573000000000000000000000000000017
:10114000000000000000000000000000004040A47B
:10115000408440844DEE52845E8450854C8600006D
:10116000000006180C30186030C0618030C0186074
:101170000C30061800000000000000000000000015
:101180000000000000000000000000000000739656
:101190004A49484949C872484A484A4871A8000023
:1011A00000000000122F12292A282948294F7D49C2
:1011B00044894489448F00000000000000000000C2
:1011C0000000000000000000000000000000739616
:1011D0004A49484949C872484A484A4871A80000E3
:1011E00000000000700050005000700007FC0FFC71
:1011F0000C000C000C000C000C000C000C000C008F
:101200000C000C000C000C000C000C000C000C007E
:101210000C000C000C000FFC07FC0000000000009C
:10122000000000007800440044004400440244E010
:101230007912410240E24012411240E200000000F7
:1012400000000000003E5B4F5B3E3E6B4F6B3E1C60
:101250003E7C3E1C183C7E3C181C577D571C1C5E77
:101260007F5E1C00183C1800FFE7C3E7FF0018244E
:101270001800FFE7DBE7FF30483A060E26297929F8
:1012800026407F050507407F05253F5A3CE73C5A2D
:101290007F3E1C1C08081C1C3E7F14227F22145F0A
:1012A0005F005F5F06097F017F006689956A606065
:1012B00060606094A2FFA29408047E040810207E5F
:1012C000201008082A1C08081C2A08081E101010E4
:1012D000100C1E0C1E0C30383E3830060E3E0E062A
:1012E000000000000000005F00000007000700147D
:1012F0007F147F14242A7F2A12231308646236493C
:101300005620500008070300001C22410000412223
:101310001C002A1C7F1C2A08083E08080080703028
:101320000008080808080000606000201008040297
:101330003E5149453E00427F40007249494946219D
:1013400041494D331814127F1027454545393C4A11
:101350004949314121110907364949493646494928
:10136000291E000014000000403400000008142270
:1013700041141414141400412214080201590906DE
:101380003E415D594E7C1211127C7F494949363EDF
:10139000414141227F4141413E7F494949417F09C5
:1013A0000909013E414151737F0808087F00417FD0
:1013B00041002040413F017F081422417F404040CE
:1013C000407F021C027F7F0408107F3E4141413E66
:1013D0007F090909063E4151215E7F0919294626E8
:1013E0004949493203017F01033F4040403F1F20EC
:1013F00040201F3F4038403F6314081463030478C3
:1014000004036159494D43007F41414102040810E2
:1014100020004141417F040201020440404040401D
:10142000000307080020545478407F28444438388B
:1014300044444428384444287F38545454180008FD
:101440007E090218A4A49C787F0804047800447DD7
:1014500040002040403D007F1028440000417F4074
:10146000007C047804787C080404783844444438C8
:10147000FC1824241818242418FC7C0804040848A8
:101480005454542404043F44243C4040207C1C20F9
:1014900040201C3C4030403C44281028444C909054
:1014A000907C4464544C44000836410000007700AE
:1014B00000004136080002010204023C2623263CBB
:1014C0001EA1A161123A4040207A38545455592146
:1014D0005555794121545478412155547840205430
:1014E0005579400C1E52721239555555593954547C
:1014F000545939555454580000457C410002457DEB
:10150000420001457C40F0292429F0F0282528F0EC
:101510007C545545002054547C547C0A097F493240
:10152000494949323248484832324A4848303A41BB
:1015300041217A3A42402078009DA0A07D39444460
:1015400044393D4040403D3C24FF2424487E4943EB
:10155000662B2FFC2F2BFF0929F620C0887E09035C
:1015600020545479410000447D413048484A323883
:101570004040227A007A0A0A727D0D19317D2629AF
:10158000292F28262929292630484D4020380808A7
:10159000080808080808382F10C8ACBA2F102834DB
:1015A000FA00007B000008142A142222142A1408CE
:1015B000AA005500AAAA55AA55AA000000FF0010CB
:1015C0001010FF00141414FF001010FF00FF101083
:1015D000F010F0141414FC001414F700FF0000FFC6
:1015E00000FF1414F404FC141417101F10101F1023
:1015F0001F1414141F00101010F0000000001F1022
:101600001010101F10101010F010000000FF10102C
:1016100010101010101010FF10000000FF14000038
:10162000FF00FF00001F10170000FC04F414141743
:1016300010171414F404F40000FF00F71414141429
:10164000141414F700F7141414171410101F101F9B
:10165000141414F4141010F010F000001F101F00E8
:1016600000001F14000000FC140000F010F0101027
:10167000FF10FF141414FF141010101F00000000BE
:10168000F010FFFFFFFFFFF0F0F0F0F0FFFFFF00B2
:1016900000000000FFFF0F0F0F0F0F3844443844C5
:1016A0007C2A2A3E147E02020606027E027E026325
:1016B000554941633844443C04407E201E200602C4
:1016C0007E020299A5E7A5991C2A492A1C4C7201A1
:1016D000724C304A4D4D303048784830BC625A46E2
:1016E0003D3E494949007E0101017E2A2A2A2A2AD3
:1016F00044445F444440514A444040444A514000BD
:1017000000FF0103E080FF000008086B6B08361241
:10171000362436060F090F060000181800000010C6
:1017200010003040FF0101001F01011E00191D17AC
:1017300012003C3C3C3C0000000000000000002384
:101740000026002900000000090003020000040533
:101750000800000000000000000000000000000081
:10176000240027002A000102040810204080010202
:1017700004081020010204081020408040000000EE
:1017800000250028002B00040404040404040402BF
:1017900002020202020303030303030202031C7E8C
:1017A00063B0C79E7E7E3E7E6730C79E7E7E7E7E15
:1017B0006730C79E7E7E62606630C79E601860603C
:1017C0006E30C79E601860606E30C79E601878608B
:1017D0006C30C7FE60187C7C7C3FC6F67C183C7C75
:1017E000783FC6F67C183E7C7C3FC6F67C180E60BF
:1017F0006C30C6F6601806606E30C6F6601806607B
:101800006E30C6F6601846606730C66660187E7E29
:101810006730C6067E187C7E6730C6067E18387E26
:1018200063B0C6067E180000000000000000000043
:1018300000000000000000000000000000000000A8
:10184000000000000000000000000000E92B11244F
:101850001FBECFEFD8E0DEBFCDBF12E0A0E0B1E009
:10186000EAE7FAE602C005900D92AE38B107D9F763
:1018700024E0AEE8B2E001C01D92A934B207E1F75E
:101880001CE0C7E2DCE004C02197FE010E94213584
:10189000C632D107C9F70E94232C0C943B350C9417
:1018A0000000CF93DF9385E090E0A0E0B0E080936C
:1018B0000E0490930F04A0931004B093110485ECD0
:1018C0009CE190930D0480930C04A0E7B0E08C9110
:1018D0008E7F8C93E0EBF0E080818C7F8083E1EB66
:1018E000F0E08081877F8083C6EBD0E088818F7DA8
:1018F00088838C918D7F8C938081846080838081AC
:101900008C7F808383E890E090930B0480930A049B
:10191000DF91CF9108952091090481E0213208F0F0
:1019200044C08091E5038111FCCF8091080492E0CE
:101930009093E50391E09093E4039FEF9093E3038A
:101940001092E2032093E103A8EEB3E0E1ECF3E0B0
:1019500090E0291331C01092C0039091C003880F0A
:10196000892B8093C0038091BF03813049F5109289
:10197000BF038091C0038093BB008091BC0083FDB6
:10198000F8CF85EC8093BC008091E5038230E1F3D1
:101990008091E3038F3FB1F08091E3038032A1F0A7
:1019A0008091E303803391F084E01092E70310927A
:1019B00009041092E60308953D9131939F5FC9CFCA
:1019C00085EEE0CF80E0F1CF82E0EFCF83E0EDCF96
:1019D00028E030E040E8E0913F04F091400450817D
:1019E00090914604909595239083E0913D04F09169
:1019F0003E0490914504582F542389F05081952B33
:101A00009083E0913F04F09140049081509146040E
:101A1000952B9083469521503109E9F60895508120
:101A200090959523EDCF81E08093BC0308950895B0
:101A30000895AF92BF92CF92DF92EF92FF920F93F1
:101A40001F93CF93DF936C017B018B01040F151F54
:101A5000EB015E01AE18BF08C017D10759F06991BC
:101A6000D601ED91FC910190F081E02DC601099520
:101A7000892B79F7C501DF91CF911F910F91FF90CD
:101A8000EF90DF90CF90BF90AF900895843081F0B9
:101A900028F4823099F08330A9F008958830A9F0B5
:101AA0008930C9F08530B1F4809180008F7D03C00A
:101AB000809180008F7780938000089584B58F7720
:101AC00084BD089584B58F7DFBCF8091B0008F7762
:101AD0008093B00008958091B0008F7DF9CFCF93AF
:101AE000DF93282F30E0F901EB5BF84E8491F90188
:101AF000EA59F84ED491F901E957F84EC491CC2334
:101B0000A1F081110E94460DEC2FF0E0EE0FFF1FB7
:101B1000E55CF84EA591B491EC91ED2381E090E065
:101B200009F480E0DF91CF91089580E090E0FACF52
:101B30001F93CF93DF93282F30E0F901EB5BF84E32
:101B40008491F901EA59F84ED491F901E957F84E18
:101B5000C491CC23A9F0162F81110E94460DEC2FC1
:101B6000F0E0EE0FFF1FE358F84EA591B4918FB748
:101B7000F894EC91111108C0D095DE23DC938FBF4F
:101B8000DF91CF911F910895DE2BF8CFCF93DF9394
:101B900090E0FC01EA59F84E24918957984EFC01D7
:101BA00084918823C9F090E0880F991FFC01E45AC2
:101BB000F84EA591B491FC01E358F84EC591D4912B
:101BC00061110DC09FB7F8948C91209582238C935E
:101BD0008881282328839FBFDF91CF9108956230A9
:101BE00051F49FB7F8943C91822F809583238C9376
:101BF000E8812E2BEFCF8FB7F894EC912E2B2C93FE
:101C00008FBFEACF3FB7F89480917C0390917D031A
:101C1000A0917E03B0917F0326B5A89B05C02F3FFE
:101C200019F00196A11DB11D3FBFBA2FA92F982F02
:101C30008827BC01CD01620F711D811D911D43E0FC
:101C4000660F771F881F991F4A95D1F708958F92C5
:101C50009F92AF92BF92CF92DF92EF92FF924B0191
:101C60005C010E94020E6B017C010E94020E6C1945
:101C70007D098E099F09683E734081059105A8F38F
:101C800021E0821A9108A108B10888EEC80E83E00D
:101C9000D81EE11CF11C81149104A104B10429F7A0
:101CA000FF90EF90DF90CF90BF90AF909F908F907C
:101CB000089508954115510529F4EAE7F0E080817F
:101CC0008F7780836A307105B9F0CB01880F991F37
:101CD000880F991F807267706860682B88E10FB663
:101CE000F894A895809360000FBE60936000E0E6D2
:101CF000F0E0808180648083232BD9F483B7817FD7
:101D0000846083BFF89483B7816083BF85B78066A2
:101D100085BF8F7D85BF7894889583B78E7F83BF7D
:101D20007894452B29F4EAE7F0E08081806880838D
:101D3000089583B7817F846083BFF89483B78160FF
:101D400083BF7894889583B78E7F83BF7894E9CFDB
:101D50000F931F93CF93DF93EC018D89823009F4A9
:101D600053C0833009F4ACC0813009F05CC0EC8111
:101D7000FD81E41BF50BAF01421B530B77FD3FC008
:101D80008E819F8168177907D4F557FF04C0240F0F
:101D9000351F50E040E08C819D81FA01E20FF31F76
:101DA0008E179F071CF49C01241B350B121613067B
:101DB00034F5FB0177FD3796A3E0F595E795AA95F5
:101DC000E1F7B6E0EE0FFF1FBA95E1F7E40FF51F5C
:101DD000ED5DFE4F6770772781E090E001C0880FCE
:101DE0006A95EAF7482F0130110509F472C008F42A
:101DF0007CC02E0F3F1F0230110509F483C0DF9114
:101E0000CF911F910F910895AC81BD81CD01861BAB
:101E1000970BBC0161507109EE81FF81E41BF50B4A
:101E2000AF01421B530B77FDEACF8C819D81681770
:101E300079072CF757FF04C0240F351F50E040E00E
:101E40008E819F81FA01E20FF31F8E179F071CF40A
:101E50009C01241B350B121613068CF6922FA42F0F
:101E6000A695A695A69580E4A89FD0011124A60F5B
:101E7000B71FAD5DBE4F477009F457C058E0541B03
:101E8000452F652F70E0FB01E55DFD4F8081251733
:101E900008F0B0C0621B71092FEF30E002C0359529
:101EA00027956A95E2F7822301301105A9F108F41C
:101EB00064C00230110509F0A2CF2C9182272EC0F8
:101EC000AE81BF81CD01861B970BBC0161507109AA
:101ED00055CF2E0F3F1FE217F30709F490CF8191E2
:101EE000DF011197842B8C93F6CF80952E0F3F1F27
:101EF000E217F30709F483CF9191DF01119798233B
:101F00009C93F6CFE217F30709F479CF8191DF01B3
:101F1000119784278C93F6CF2C91822B8C93941756
:101F200008F46DCF941BA05CBF4F983008F447C0F5
:101F30000230110531F5FD01892F20812095208384
:101F4000E05CFF4F88508830C0F728EF290F2695B6
:101F50002695269530E02F5F3F4F86E0220F331FF6
:101F60008A95E1F7A20FB31F977009F448CFE92FC4
:101F7000F0E0ED5DFD4F808132C080952C91822391
:101F8000CDCF81E00130110509F080E08195FD01A0
:101F9000292F8083E05CFF4F28502830D0F728EFAE
:101FA000290F26952695269530E02F5F3F4F46E076
:101FB000220F331F4A95E1F7A20FB31F97709923A1
:101FC00009F41DCFE92FF0E0ED5DFD4F8081013078
:101FD000110541F058F00230110509F010CF9C9125
:101FE000892702C09C91892B8C9309CF80959C9165
:101FF0008923FACF0130110509F48ECF08F4BDCF43
:102000000230110509F459CF8DCF0F931F93CF9351
:10201000DF93EC018D89823009F45EC0833009F4CE
:10202000B5C0813009F067C0AC81BD81CD01841B92
:10203000950BAC014150510957FD49C08C819D81E0
:10204000481759070CF043C077FF04C0260F371F0D
:1020500070E060E08E819F81FB01E20FF31F8E171D
:102060009F071CF49C01261B370B121613067CF5E8
:10207000922FA62FA695A695A69580E4A89FD0019D
:102080001124A40FB51FAD5DBE4F677009F48FC05A
:1020900048E0461B642F70E0FB01E55DFD4F808149
:1020A000241708F002C1621B71092FEF30E002C053
:1020B000359527956A95E2F782230130110509F4D9
:1020C0006DC008F49CC00230110509F4F8C0DF911E
:1020D000CF911F910F910895EC81FD81E61BF70BC5
:1020E000AE81BF81CD01841B950BAC0141505109DC
:1020F000BF01621B730B57FDEACF8E819F8148178A
:1021000059072CF777FF04C0260F371F70E060E0F7
:102110008C819D81FB01E20FF31F8E179F071CF43A
:102120009C01261B370B121613068CF6FA0157FD7D
:10213000379693E0F595E7959A95E1F7A6E0EE0FCF
:10214000FF1FAA95E1F7E60FF71FED5DFE4F477001
:10215000552781E090E001C0880F4A95EAF7482FA3
:102160000130110509F488C008F492C02E0F3F1FFA
:102170000230110509F0ABCFE217F30709F4A7CF3E
:102180008191DF01119784278C93F6CFEE81FF8137
:10219000E61BF70BBF01621B730B4ECF2C91822BFA
:1021A0008C93941708F493CF941BA05CBF4F983086
:1021B00008F447C00230110531F5FD01892F208157
:1021C00020952083E05CFF4F88508830C0F728EFCF
:1021D000290F26952695269530E02F5F3F4F86E004
:1021E000220F331F8A95E1F7A20FB31F977009F4EE
:1021F0006ECFE92FF0E0ED5DFD4F808132C080951C
:102200002C918223CDCF81E00130110509F080E0CF
:102210008195FD01292F8083E05CFF4F28502830F5
:10222000D0F728EF290F26952695269530E02F5FC9
:102230003F4FC6E0220F331FCA95E1F7A20FB31F2D
:102240009770992309F443CFE92FF0E0ED5DFD4F3E
:1022500080810130110541F058F00230110509F07C
:1022600036CF9C91892702C09C91892B8C932FCFCC
:1022700080959C918923FACF2E0F3F1FE217F30719
:1022800009F425CF8191DF011197842B8C93F6CF30
:1022900080952E0F3F1F2E173F0709F418CF9191FD
:1022A000DF01119798239C93F6CF0130110509F4B3
:1022B00075CF08F4A4CF0230110509F075CF2C9129
:1022C00082276ECFDC0177FD67C018968D919C91B7
:1022D0001997681779070CF05FC057FD5DC01A9613
:1022E0008D919C911B97481759070CF055C0559636
:1022F0008C9155978230B9F0833041F1813049F4A7
:1023000014968D919C91841B950BAB01BC0161507F
:1023100071092130310521F108F43FC02230310527
:1023200009F458C008951496ED91FC911597E61B99
:10233000F70BBF016150710916968D919C91FC01BC
:10234000E41BF50BAF0141505109E3CF16968D9177
:102350009C91861B970BBA01AC0141505109D9CF12
:10236000FA0157FD3796A3E0F595E795AA95E1F7B1
:10237000B6E0EE0FFF1FBA95E1F7E60FF71FED5D30
:10238000FE4F4770552721E030E001C0220F4A95EB
:10239000EAF78081822B80830895FA0157FD3796F2
:1023A00023E0F595E7952A95E1F736E0EE0FFF1F5C
:1023B0003A95E1F7E60FF71FED5DFE4F47705527A1
:1023C00081E090E001C0880F4A95EAF780959081FE
:1023D0008923E1CFFA0157FD379683E0F595E7951C
:1023E0008A95E1F796E0EE0FFF1F9A95E1F7E60F69
:1023F000F71FED5DFE4F4770552721E030E001C02B
:10240000220F4A95EAF780818227C5CF2F923F920B
:102410004F925F926F927F928F929F92AF92BF92F4
:10242000CF92DF92EF92FF920F931F93CF93DF93A0
:1024300000D000D0CDB7DEB73C014A0159016B8313
:102440007C83C90107969C0193E0359527959A9561
:10245000E1F73A8329832B803C80200E311ED12C5A
:10246000C12C270131E0432610E000E0F80183E0B1
:10247000F595E7958A95E1F7EC0DFD1DE80DF91D41
:10248000E491B801660D771DC8018770992720E88F
:1024900030E002C0359527958A95E2F7C901F0E052
:1024A000E223F9239701EF2B09F492014B815C8120
:1024B0008EE194E00E9462110F5F1F4FA016B106DB
:1024C000A9F68B819C8101969C838B8329813A811B
:1024D000C20ED31E2816390639F60F900F900F90B2
:1024E0000F90DF91CF911F910F91FF90EF90DF90B0
:1024F000CF90BF90AF909F908F907F906F905F90A4
:102500004F903F902F90089508952F923F924F92B1
:102510005F926F927F928F929F92AF92BF92CF9273
:10252000DF92EF92FF920F931F93CF93DF93CDB77C
:10253000DEB72C970FB6F894DEBF0FBECDBF9C83DD
:102540008B836A3061F5DC0154968C91B8E08B9FE7
:1025500090011124EB81FC8186859785820F931F62
:10256000978786871586148681E090E02C960FB6B3
:10257000F894DEBF0FBECDBFDF91CF911F910F91B9
:10258000FF90EF90DF90CF90BF90AF909F908F9093
:102590007F906F905F904F903F902F9008956D3097
:1025A00019F32B813C813C872B87D9011C96CD9058
:1025B000DC901D9718968D919C911997C816D90695
:1025C0000CF07FC01E968D909C901F971A968D914F
:1025D0009C911B97881699060CF073C05496BC9179
:1025E000B983AB2EB12CC601E6E0BE9F800D911DD4
:1025F0001124181619060CF064C0C50143E0880FB9
:10260000991F4A95E1F7880D991D181619060CF0C7
:1026100058C0D90152960D90BC91A02DBC83AB83BC
:10262000F9010088F189E02DFE83ED83F5E06F9FCD
:10263000B001112426011A826C197D099B01205CCE
:102640003D4E3A8729873A81E0E0353029F0E98527
:10265000FA85E40DF51DE4911401712C612C8E2F87
:1026600090E098878F83E0FF6AC0AB85BC85ED91D1
:10267000FC91B981B13009F055C00480F581E02D9D
:102680002D813E81A401460D571DB2018B859C858D
:102690000995EF81F885F595E795FFEF6F1A7F0AA9
:1026A0002A0C3B1C28E062167104C9F63FEF431A5E
:1026B000530ACA0CDB1C5A815F5F5A83563009F0FB
:1026C000C2CFAB85BC8554964C915497242F30E0F3
:1026D0001C968D919C91B6E04B9F800D911D11240D
:1026E000EB85FC85958784874689442309F43CCF94
:1026F0006AEF6203A001639F500D1124608571850C
:10270000460F571F481759070CF02ECF83E0220FB2
:10271000331F8A95E1F786859785280F391F3787FC
:10272000268720CF0684F785E02DED80FE80850189
:102730009501A101B6018B859C850995AACFEB81F6
:10274000FC812D813E81E217F30709F4A2CFAB850E
:10275000BC85ED91FC91B981B13031F40480F581F3
:10276000E02D2B813C818ECF0684F785E02DEB8018
:10277000FC80DDCFEF92FF920F931F93DC011A963E
:102780000D911C911B9718962D913C911997ED91E5
:10279000FC910684F785E02D7B0150E040E070E07D
:1027A00060E009951F910F91FF90EF9008956F924F
:1027B0007F928F929F92AF92BF92CF92DF92EF92D1
:1027C000FF920F931F93CF93DF936C015A0148013F
:1027D000EB013B01620E731EC615D70574F4D601DA
:1027E000ED91FC910084F185E02D87019401A50114
:1027F000BE01C60109952196EFCFDF91CF911F91C0
:102800000F91FF90EF90DF90CF90BF90AF909F908F
:102810008F907F906F900895EF92FF920F931F9388
:10282000260F371F21503109DC01ED91FC91068004
:10283000F781E02D78018A0109951F910F91FF9092
:10284000EF900895EF92FF920F931F93240F351F7F
:1028500021503109DC01ED91FC910680F781E02DDA
:10286000780189019B0109951F910F91FF90EF90CD
:1028700008956F927F928F929F92AF92BF92CF9264
:10288000DF92EF92FF920F931F93CF93DF93EC01B0
:102890006B015A0139014801E881F9810284F3850D
:1028A000E02D87010995A501480D591D4150510999
:1028B000E881F9810284F385E02D9301B601CE0110
:1028C0000995E881F9810084F185E02D9401A50145
:1028D000B601CE010995C60CD71CB601615071092D
:1028E000E881F9810084F185E02D9401A501CE01F4
:1028F0000995DF91CF911F910F91FF90EF90DF909D
:10290000CF90BF90AF909F908F907F906F900895E1
:102910002F923F924F925F926F927F928F929F92EF
:10292000AF92BF92CF92DF92EF92FF920F931F93DD
:10293000CF93DF9300D000D000D0CDB7DEB73C01FD
:102940006A013E832D83FC82EB825801A41AB50AEA
:10295000B7FE03C0B194A194B1088D809E80861A01
:10296000970A97FE03C09194819491088A149B045E
:102970005CF0902F812F0D811E819D838E839C2D75
:102980008D2D6B01692F782F0C151D055CF09D8135
:102990008E817E836D83692F782F902F812F860102
:1029A000C92ED82E1601201A310A2B012D813E8105
:1029B000421A530A57FE03C05194419451087101C1
:1029C00037FE03C03FEFE31AF30AF594E7948D81D5
:1029D0009E81861797075CF5A1E0B0E0BA83A983D2
:1029E000C016D1064CF1D301ED91FC910480F58124
:1029F000E02D2B813C81A8016D817E818A149B048E
:102A00001CF04D815E81B801C3010995E418F508F9
:102A1000F7FE0AC02D813E8189819A81280F391FD6
:102A20003E832D83E20CF31C0F5F1F4FD9CF2FEF96
:102A30003FEF3A832983D4CF26960FB6F894DEBFB2
:102A40000FBECDBFDF91CF911F910F91FF90EF90FF
:102A5000DF90CF90BF90AF909F908F907F906F90BE
:102A60005F904F903F902F900895DF92EF92FF92EA
:102A70000F931F93CF93DF93D62EC82FD0E0DC1691
:102A800078F0EE24E394F12C0EE010E09E0144E097
:102A900050E0BE018EE194E00E9488142196EFCFB1
:102AA000DF91CF911F910F91FF90EF90DF900895EC
:102AB00085ED8093BC008091BC0084FDFCCF10921A
:102AC000E503089520915403260F3327331F213245
:102AD0003105ECF42091E503FC0190E080E0243026
:102AE00069F082E00895A09154032191AC014C5CFF
:102AF0005C4FA40FB52FB11D2C930196861798F348
:102B000080915403680F6093540380E0089581E03E
:102B100008950895E0918D0380918C03E81730F4B7
:102B2000F0E0EC5EFC4F808190E008958FEF9FEF26
:102B3000089590918D0380918C032FEF3FEF9817AC
:102B400048F4E92FF0E0EC5EFC4F208130E09F5F1D
:102B500090938D03C901089580918C0390918D030A
:102B6000891B990B0895CF92DF92EF92FF920F93FA
:102B70001F93CF93DF937C01CB018A012091E60361
:102B8000222389F0EB016B01C40ED51ECC15DD05A7
:102B900069F06991D701ED91FC910190F081E02DF0
:102BA000C7010995F3CF642F0E946215C801DF9118
:102BB000CF911F910F91FF90EF90DF90CF900895EC
:102BC000CF93DF931F92CDB7DEB769832091E603E1
:102BD0002223F9F020910904203258F021E030E05E
:102BE000FC013383228390E080E00F90DF91CF914E
:102BF00008958091E703E82FF0E0E851FC4F9981B8
:102C000090838F5F8093E7038093090481E090E0D5
:102C1000ECCF61E0CE0101960E946215F7CFCF9311
:102C2000C82F809137048F3FB1F1E0914104F091BA
:102C30004204808190914704892B8083E091430472
:102C4000F091440490818091480480958923808389
:102C5000E0914104F0914204908180914704809575
:102C60008923808380913C04882389F0CEBD0000B5
:102C70000DB407FEFDCF8EB5E0914104F091420402
:102C8000808190914704892B8083CF9108958C2F68
:102C90000E94E80CF1CF8091350491E09093E60317
:102CA000809308041092E7031092090460E082E127
:102CB00094E00E94E0156C2F82E194E00E94E01500
:102CC000CF910C948B0C8FEA0E940F161092BE03CA
:102CD0001092BD030895DF92EF92FF920F931F931E
:102CE000CF93DF9381E20E940F1680E20E940F16BD
:102CF0008FE50E940F1682E20E940F1680E00E946C
:102D00000F1683E00E940F16809137048F3F09F45D
:102D100042C0E0914104F0914204808190914704C7
:102D2000892B8083E0914304F09144048081909149
:102D30004804892B8083E0914104F0914204908102
:102D400080914704809589238083C3E2D1E003E228
:102D500012E0899190913C049923D1F08EBD00003E
:102D60000DB407FEFDCF8EB50C171D0791F7E0914E
:102D70004104F0914204808190914704892B808323
:102D8000DF91CF911F910F91FF90EF90DF90089509
:102D90000E94E80CE9CF0091B8008CE08093B80065
:102DA000C3E2D1E0DD24D39480913504D092E603D0
:102DB000809308041092E7031092090460E482E112
:102DC00094E00E94E0157E0110E1F70161917F011E
:102DD00082E194E00E94E0151150B9F70E948B0C3B
:102DE0006096F2E0C332DF07F9F60093B800C8CF6F
:102DF00010921003109211031092120310921303F9
:102E000010920F0380910A0490910B048093B200FA
:102E1000E0E7F0E08081816080830895EF92FF9287
:102E20000F931F93EE24E394F12C00E110E020E1D6
:102E300030E040E252E160E170E080E390E00E9427
:102E400006121F910F91FF90EF9008958F929F921D
:102E5000AF92BF92CF92DF92EF92FF920F931F93A8
:102E6000CF93DF934B015C0180911401882309F417
:102E7000A5C020E030EC49E754E4C5010E945A3473
:102E800018163CF4812C80EC982E89E7A82E84E457
:102E9000B82EC501B4010E947233FB01CB0164E678
:102EA00070E00E94CC349B01CAE0D0E0BE010E94D9
:102EB000CC346B01CF01BE010E94CC34EC01222343
:102EC000B1F0A901552716E0440F551F1A95E1F7F7
:102ED000405A514FEE24E394F12C00E210E020E13F
:102EE00030E070E060E090E080E00E940612A60111
:102EF0005527A6E0440F551FAA95E1F7405A514FB8
:102F0000EE24E394F12C00E210E020E130E070E0E8
:102F100060E080E190E00E940612AE015527C6E015
:102F2000440F551FCA95E1F7405A514F20E130E058
:102F300070E060E081E290E00E9406128EE18093F2
:102F400012018AE180931101C0901101D12CC0912E
:102F50001201D0E04E018FEF881A980A21E030E08C
:102F6000A601B4018EE194E00E94621156018FEF38
:102F7000A81AB80A21E030E0A501B4018EE194E07E
:102F80000E94621121E030E0A601BE018EE194E0D2
:102F90000E94621121E030E0A501BE018EE194E0C3
:102FA000DF91CF911F910F91FF90EF90DF90CF9025
:102FB000BF90AF909F908F900C94621121E73FE0FB
:102FC00048E651E4C5010E945F344B015C0120E0FA
:102FD0003CE34CE156E40E945A3418163CF4812C30
:102FE000FCE39F2EFCE1AF2EF6E4BF2EC501B40139
:102FF0000E9472339B01CB0168EE73E00E94CC34D7
:10300000FB0104E610E0B8010E94CC34EB01C901D9
:10301000B8010E94CC340AE010E0B8010E94CC3420
:103020005B01C901B8010E94CC346C014F019924A5
:10303000EE23A9F0A40176E0440F551F7A95E1F73D
:10304000405E594FEE24E394F12C00E210E020E1C1
:1030500030E070E060E090E080E00E940612AE0197
:103060005527840E951E8928A1F036E0440F551F80
:103070003A95E1F7405E594FEE24E394F12C00E2DB
:1030800010E020E130E070E060E08CE090E00E9431
:103090000612A501552786E0440F551F8A95E1F7D2
:1030A000405E594FEE24E394F12C00E210E020E161
:1030B00030E070E060E088E190E00E940612A60136
:1030C000552726E0440F551F2A95E1F7405E594FDA
:1030D00020E130E070E060E086E290E00E940612BD
:1030E00083E28093120189E12DCFEF92FF920F933B
:1030F0001F930E942617EE24E394F12C00E210E0C7
:1031000020E130E040EA51E170E060E081E390E0EE
:103110000E94061280911401811106C01F910F9127
:10312000FF90EF900C940E171F910F91FF90EF906E
:103130000895EF92FF920F931F930E942617EE249B
:10314000E394F12C00E210E020E130E040E651E1B0
:1031500070E060E081E390E00E940612809114012B
:10316000811106C01F910F91FF90EF900C940E17E4
:103170001F910F91FF90EF9008958F929F92AF92C1
:10318000BF92CF92DF92EF92FF920F931F93CF9354
:10319000DF936B017C0180911401882309F47CC0CA
:1031A00020E030EC49E754E4C7010E945A34181675
:1031B0003CF4C12C90ECD92E99E7E92E94E4F92E39
:1031C000C701B6010E9472339B01CB0164E670E037
:1031D0000E94CC34FB010AE010E0B8010E94CC341C
:1031E000EB01C901B8010E94CC346C015F01BB2422
:1031F000EE23A9F0A50106E0440F551F0A95E1F75B
:10320000405A514FEE24E394F12C00E210E020E10B
:1032100030E070E060E090E080E00E940612AE01D5
:103220005527A40EB51EAB28A1F0D6E0440F551FBC
:10323000DA95E1F7405A514FEE24E394F12C00E285
:1032400010E020E130E070E060E080E190E00E947A
:103250000612A6015527B6E0440F551FBA95E1F7AF
:10326000405A514FEE24E394F12C00E210E020E1AB
:1032700030E070E060E080E290E00E940612DF91B2
:10328000CF911F910F91FF90EF90DF90CF90BF9063
:10329000AF909F908F9008958091B303853049F04F
:1032A00021E73FE048E651E4C7010E945F346B012B
:1032B0007C0120E03CE34CE156E4C701B6010E94EA
:1032C0005A3418163CF4C12CACE3DA2EACE1EA2EE9
:1032D000A6E4FA2EC701B6010E9472339B01CB010E
:1032E00068EE73E00E94CC34FB01C4E6D0E0BE017E
:1032F0000E94CC345B01C901BE010E94CC340AE0BB
:1033000010E0B8010E94CC34EB01C901B8010E9461
:10331000CC346C014F019924EE23A9F0A401E6E01E
:10332000440F551FEA95E1F7405E594FEE24E394B0
:10333000F12C00E210E020E130E070E060E090E08D
:1033400080E00E940612A50155275A01A80CB91C5D
:10335000A114B104A1F066E0440F551F6A95E1F78E
:10336000405E594FEE24E394F12C00E210E020E19E
:1033700030E070E060E08CE090E00E940612AE0168
:103380005527A40EB51EAB28A1F026E0440F551F0B
:103390002A95E1F7405E594FEE24E394F12C00E2C8
:1033A00010E020E130E070E060E088E190E00E9411
:1033B0000612A601552786E0440F551F8A95E1F7AE
:1033C000405E594FEE24E394F12C00E210E020E13E
:1033D00030E070E060E084E290E04FCFEF92FF9247
:1033E0000F931F93BC01990F880B990B0E94AA336E
:1033F00020911401211106C021E73FE048E651E485
:103400000E9400330E94BD18EE24E394F12C00E2E8
:1034100010E020E130E040E251E170E060E080E364
:1034200090E00E9406121F910F91FF90EF90089577
:10343000CF92DF92EF92FF928091130120E4829F5E
:10344000C0011124826080937C0080917A008064A6
:1034500080937A0080917A0086FDFCCF809178007D
:1034600060917900762F682F072E000C880B990B3E
:103470000E94AA3324E63AE345E95BE30E945F3405
:103480006B017C0123E333E343E550E40E948E3279
:1034900025E83BEE41E55FE30E94003320E030E0A9
:1034A00048EC52E40E945F340E9472336536710525
:1034B000DCF470930E0360930D0320E030E040E8ED
:1034C00050E4C701B6010E945A341816A4F48FEFD5
:1034D00090E09093B6038093B5031092B003FF90F1
:1034E000EF90DF90CF90089584E690E090930E03E4
:1034F00080930D03E2CF26E636E646E650E4C701A8
:10350000B6010E945A3418161CF482E890E0E1CF0C
:1035100023E333E343E550E4C701B6010E945A3484
:10352000181674F41092B6031092B5038091B0038C
:10353000882311F0833099F681E08093B003CFCFD8
:1035400020E030E0A901C701B6010E945A341816E4
:1035500034F610922201C3CF1F93CF93DF93909143
:103560009503992341F0981731F0C0E08C2FDF913B
:10357000CF911F9108951091AF031130B1F7D82F5B
:103580000E946F0DC82F80919003C1112CC0811132
:10359000AAC06AE070E080E090E00E94270E8D2FC4
:1035A0000E946F0DC82F81110FC0D0939503109307
:1035B00090038091B1039091B2038130910521F481
:1035C0009093FC028093FB0280919003813069F616
:1035D000C111CBCF8091A503813039F61092A5039C
:1035E0001092A203C3CF813079F7C13069F0809186
:1035F000B1039091B203019739F78091F90290914C
:10360000FA02883C910504F38091FB029091FC0240
:10361000019779F48091F9029091FA02873C910523
:1036200044F41092FC021092FB021092FA021092E3
:10363000F9028091FB029091FC02029769F51092C9
:10364000A503C13051F41092FC021092FB021092BB
:103650009503109290031092A203809120010E9482
:103660006F0D892B09F0B0CF8091B303893009F039
:10367000ABCFD33009F0A8CF8091090390910A0312
:10368000181619060CF4A0CF83E090E09093FC028A
:103690008093FB02C3E06ACF8091B1039091B203A3
:1036A0000197B9F48091F9029091FA02883C910552
:1036B00084F01092A5031092A20382E090E0909310
:1036C000FC028093FB021092FA021092F902C2E00F
:1036D0004DCF10929503109290031092A503109273
:1036E000A203C1E043CF813009F06ECF80CF4F926B
:1036F0005F926F927F928F929F92AF92BF92CF9282
:10370000DF92EF92FF92409080035090810360908F
:10371000820370908303C0908403D0908503E0906F
:103720008603F0908703C418D508E608F708C70198
:10373000B6010E94A8334B015C018092F502909281
:10374000F602A092F702B092F802AAEFB0E0A3014D
:1037500092010E9402350E94A833A50194010E94A3
:10376000003320E030E048E452E40E948E3260935F
:10377000F1027093F2028093F3029093F402A8E7AF
:10378000B0E0A70196010E9402352AEF30E040E048
:1037900050E00E94E0342093ED023093EE0240931B
:1037A000EF025093F002FF90EF90DF90CF90BF9028
:1037B000AF909F908F907F906F905F904F90089503
:1037C00061E08FE00E94980D60E08FE00C94980D0E
:1037D00061E08DE00E94980D61E08FE00E94C60DCF
:1037E00060E08EE00E94C60D0C94E01BCF938091A8
:1037F00022018F3FD1F40E94510C0E94F8161092C2
:103800009203C1E0C093220182E080939103109261
:10381000A50310929003109295030E94E81B8091DB
:10382000A403833011F4C093A403CF910895FC0145
:1038300001900020E9F73197AF01481B590BBC01FB
:103840008EE194E00C94190D8F929F92AF92BF92EB
:103850000F931F93CF93DF93CDB7DEB7A1970FB62A
:10386000F894DEBF0FBECDBF19A2423008F44AE083
:103870008E010F5D1F4F842E912CB12CA12CA50120
:1038800094010E94E034E62FB901CA01EA30F4F451
:10389000E05DD801EE938D01232B242B252B79F7A6
:1038A00090E080E0109719F0CD010E94171CA196BE
:1038B0000FB6F894DEBF0FBECDBFDF91CF911F9141
:1038C0000F91BF90AF909F908F900895E95CE1CFEA
:1038D000CF92DF92EF92FF92CF93DF936B017C0147
:1038E0006DE28EE194E00E948512EC016627772755
:1038F000CB016C197D098E099F094AE00E94241CA6
:103900008C0F9D1FDF91CF91FF90EF90DF90CF90B4
:103910000895EEE1F4E0648B61E070E0738B628BFC
:10392000718B608B55874487378726870E94171CC9
:103930008BE592E00E94171C08958093320481E089
:1039400090E0909331048093300490932F048093FF
:103950002E0470932B0460932A0450932D044093FB
:103960002C04B901330F880B990B97FD0C94681C3C
:103970004AE00C94241CBC01990F880B990B97FD0D
:103980000C94681C4AE00C94241C4F925F926F9236
:103990007F928F929F92AF92BF92CF92DF92EF92DF
:1039A000FF920F931F93CF93DF9300D000D000D0EE
:1039B000CDB7DEB72091B9033091BA032F5F3F4FE7
:1039C0003A8329833093BA032093B9038091FB0291
:1039D0009091FC02019749F48091F9029091FA02CA
:1039E00001969093FA028093F9028091F9029091E6
:1039F000FA02893C910534F088EC90E09093FA0249
:103A00008093F90280912201823079F48091A2039F
:103A100081110BC01092EC021092EB021092EA029C
:103A20001092E90281E08093A2038091A203813089
:103A300049F48091E9029091EA0201969093EA029A
:103A40008093E9028091E9029091EA02813E9E42D0
:103A50006CF08091EB029091EC0201969093EC0255
:103A60008093EB021092EA021092E90220910D017C
:103A700030910E018091EB029091EC028217930736
:103A8000B4F01092E8021092E7021092EC02109249
:103A9000EB0284E190E090931E0180931D0110924F
:103AA00022011092EA021092E9021092AF03809173
:103AB0002201813039F484E0809322011092B40312
:103AC0000E94181A8091BD039091BE03019759F48A
:103AD00049815A814039514031F40E94181A10929C
:103AE000BA031092B90380912201823009F082C298
:103AF0008091A503811107C01092E6021092E502A1
:103B000081E08093A5032091A503213049F48091A1
:103B1000E5029091E60201969093E6028093E50219
:103B20008091E5029091E60260910B0170910C0189
:103B300038EC369FA001379F500D112448175907C4
:103B40002CF4213019F422E02093A5032091E70200
:103B50003091E802232B41F4CD9734F081E090E0DE
:103B60009093E8028093E7028091E7029091E80247
:103B7000019749F48091E3029091E40201969093B9
:103B8000E4028093E3028091E3029091E402C29701
:103B90000CF430C2009192030D83C12CD12C76011C
:103BA00001113AC0809191038230A1F410929103E7
:103BB0001092CD021092CE021092CF021092D0023B
:103BC0001092C9021092CA021092CB021092CC023B
:103BD0001092C8020091C80209830A30ACF48091A7
:103BE0009103811104C060E08FE00E94980D8EE087
:103BF0000E946F0D892B09F414C281E08093910318
:103C00000981063009F466C2C0909402D0909502F2
:103C1000E0909602F090970280919203813009F033
:103C2000E9C12091A6033091A7034091A8035091C8
:103C3000A90329833A834B835C83C092A603D09265
:103C4000A703E092A803F092A903109292031092A6
:103C5000E4021092E302C701B6010E948E324B01CA
:103C60005C012091DF023091E0024091E10250912D
:103C7000E2020E948F322B013C0120E030E048EC50
:103C800052E40E945A3418160CF4C5C34092DF0265
:103C90005092E0026092E1027092E20220E030E095
:103CA00040E450E46091DF027091E0028091E10213
:103CB0009091E2020E945A34181694F420E030E009
:103CC00040E85EE3C501B4010E94FB3287FF08C0F3
:103CD0001092DF021092E0021092E1021092E202D2
:103CE0004091AA035091AB035E834D83423051054E
:103CF0000CF466C0A70196016091DB027091DC02B2
:103D00008091DD029091DE020E948E3220E030E050
:103D100040E251E40E945F344B015C016D817E8181
:103D200061507109072E000C880B990B0E94AA3371
:103D30009B01AC01C501B4010E9400334B015C0141
:103D400020E030E0A9010E94FB3287FD6DC3809224
:103D5000960390929703A0929803B0929903609172
:103D6000090170910A01072E000C880B990B0E9423
:103D7000AA339B01AC01C701B6010E948E3220918B
:103D800096033091970340919803509199030E94B4
:103D9000003320E030E040E251E40E945F344B0108
:103DA0005C0120E030E0A9010E94FB3287FD45C3A1
:103DB00080929E0390929F03A092A003B092A103D1
:103DC0008090DF029090E002A090E102B090E202C9
:103DD0008091AC0318167CF420E030E040E251E41E
:103DE000C501B4010E945A3418162CF482E0809365
:103DF000AC031092A50380919403823009F477C03C
:103E000020E030E040E251E4C501B4010E945A34A0
:103E100018160CF048C08D819E81892BA1F060910D
:103E2000D9027091DA02072E000C880B990B0E94C0
:103E3000AA33A50194010E948F320E9472337093BD
:103E4000DA026093D9028091D9029091DA024E97FA
:103E500044F11092DA021092D9021092AB03109240
:103E6000AA0310929A0310929B0310929C03109243
:103E70009D0310929603109297031092980310924C
:103E8000990310929E0310929F031092A003109228
:103E9000A1031092DF021092E0021092E102109250
:103EA000E2021092A2038091D9029091DA02892B4A
:103EB00049F08091D7029091D80201969093D80250
:103EC0008093D7028091D7029091D802803E914092
:103ED00034F48091AA039091AB03892B41F41092A2
:103EE000D8021092D7021092DA021092D9020091F1
:103EF000A3030D836091DF027091E0028091E102E3
:103F00009091E2029058209101013091020140917C
:103F10000301509104010E945A34181614F400232E
:103F200021F00D81013009F065C08091D50290919A
:103F3000D602009761F429813A814B815C812093FC
:103F4000D1023093D2024093D3025093D40201960F
:103F50009093D6028093D50221E02093A303109280
:103F6000A2032091A503233011F01092A503209104
:103F70000001022E000C330B8217930799F5109263
:103F8000A3031092D6021092D502A7019601609168
:103F9000D1027091D2028091D3029091D4020E94FA
:103FA0008E3220E030E040E251E40E945F346093C2
:103FB0009A0370939B0380939C0390939D0380913D
:103FC000AA039091AB0301969093AB038093AA034D
:103FD000019741F4C092DB02D092DC02E092DD0254
:103FE000F092DE021092DF021092E0021092E102E3
:103FF0001092E20226960FB6F894DEBF0FBECDBF38
:10400000DF91CF911F910F91FF90EF90DF90CF90B4
:10401000BF90AF909F908F907F906F905F904F90E8
:1040200008951092910318E10E94E01B8EE00E9417
:104030006F0D4091CD025091CE026091CF027091F0
:10404000D002892B09F444C041604093CD025093C3
:10405000CE026093CF027093D002C090CD02D09078
:10406000CE02E090CF02F090D002CC0CDD1CEE1C12
:10407000FF1CC092CD02D092CE02E092CF02F0920D
:10408000D002115089F60E94E01B0E94E01B0E94A2
:10409000E01BC092C902D092CA02E092CB02F09219
:1040A000CC021092CD021092CE021092CF0210924A
:1040B000D002098124E00202F0011124E056FD4FF4
:1040C000C082D182E282F3820F5F0093C80282CD68
:1040D0004E7FBBCF2091A0023091A1024091A2025D
:1040E00049831091A302E0EAF2E0C12CD12C7601C1
:1040F00080E090E0DC0140E050E0BA0181909190D6
:10410000A190B1900D81002309F431C18416950668
:10411000A606B70608F032C188169906AA06BB069D
:1041200010F4D501C401C80CD91CEA1CFB1C0D817C
:104130000F5F0D83063011F7C41AD50AE60AF70A95
:10414000C81AD90AEA0AFB0A82E0F694E794D794DF
:10415000C7948A95D1F780919403823009F489C07D
:1041600080912101863009F06BC020E8C21626E953
:10417000D20628E9E206F10408F062C0C0929C026F
:10418000D0929D02E0929E02F0929F02409198028E
:104190005091990260919A0270919B024C155D05B5
:1041A0006E057F0570F446015701841A950AA60A28
:1041B000B70A8092900290929102A0929202B092DD
:1041C0009302C416D506E606F70670F44A015B01B1
:1041D0008C189D08AE08BF088092900290929102C0
:1041E000A0929202B092930240909002509091025D
:1041F00060909202709093028090ED029090EE0297
:10420000A090EF02B090F00284149504A604B704C5
:1042100008F0B7C020918E0230918F022F5F3F4F80
:1042200030938F0220938E022630310509F0AEC004
:10423000C0929802D0929902E0929A02F0929B0268
:104240009FEF980F953008F0A4C030E8C31636E908
:10425000D30638E9E306F10408F09BC0C092980247
:10426000D0929902E0929A02F0929B028F5F809323
:1042700021018091090390910A031816190694F5FB
:104280008230910509F092C080910501909106015C
:10429000DC011197BA83A9831B9720F50B97E1F0F6
:1042A000C701B6012AE030E040E050E00E94E0346F
:1042B0008091050390910603A0910703B091080334
:1042C000820F931FA41FB51F8093050390930603CD
:1042D000A0930703B093080329813A813093060124
:1042E00020930501AAEFB0E0A70196010E940235D4
:1042F0000E94A8332091F5023091F6024091F70216
:104300005091F8020E9400332091F1023091F202A4
:104310004091F3025091F4020E948E326B017C01B5
:10432000C0929402D0929502E0929602F092970287
:104330001092C80281E0809392030E94E01B20E06B
:1043400030E048EC51E4C701B6010E945A34181617
:1043500054F420E030E048EC53E4C701B6010E9479
:10436000FB3287FD59CCC12CD12C76015ACCC90126
:10437000A981B12FA9016A2F712FD5CEB501A40152
:10438000D2CE10928F0210928E0252CF6A017B0120
:104390004FCF41E0C41644E2D40644EFE406F104F2
:1043A00008F467CFC12CD12C760163CF039709F0B5
:1043B00099CF8091050190910601AC0141505109BE
:1043C0005A8349834B30510508F08CCF0B97E1F0AD
:1043D000C701B6012AE030E040E050E00E94E0343E
:1043E0008091010390910203A0910303B091040313
:1043F000820F931FA41FB51F8093010390930203A4
:10440000A0930303B093040389819A8190930601DA
:104410008093050167CF1092DF021092E0021092A4
:10442000E1021092E2023ACC1092960310929703A6
:10443000109298031092990392CC10929E031092BE
:104440009F031092A0031092A103BACCE3E2F1E023
:1044500080E091E0DF019C011D9221503040E1F7A6
:104460000895EF92FF920F931F93CF93DF93EA018A
:104470000E94BD1880911401EE24E394F12C88234E
:1044800009F493C000E210E020E130E040EE50E19A
:1044900070E060E080E390E00E9406129E0150E030
:1044A00040E060E370E081E090E00E949D1C83E0CA
:1044B0000E946F0D892B09F071C01092A5030E9414
:1044C0002622EE24E394F12C0BE110E025E330E00A
:1044D00044E150E065E370E08EE194E00E948814CE
:1044E00024E330E044E150E064E370E08EE194E0E6
:1044F0000E94881400E110E028E230E040E150E042
:104500006CE070E08EE194E00E94391420910D037C
:1045100030910E0342E150E066E170E0243631054F
:1045200031F424E630E042E150E06EE070E082E0F9
:1045300090E00E949D1C80911F010E946F0D892BAD
:1045400069F51092AB031092AA0310929A0310928D
:104550009B0310929C0310929D031092960310925D
:104560009703109298031092990310929E03109251
:104570009F031092A0031092A1030E942622EE2412
:10458000E394F12C00E110E020E430E040EE5CE048
:1045900070E060E090E080E00E940612DF91CF9131
:1045A0001F910F91FF90EF90089500E110E020E13E
:1045B00030E040E252E160E170E06CCF0E943635BD
:1045C0004F925F926F927F928F929F92AF92BF9223
:1045D000CF92DF92EF92FF920F931F93CF93DF93CF
:1045E0008091AD0381112AC083E00E94AC1A813012
:1045F00009F00BC19091B30391110CC08093AD03EE
:1046000080919403082E000C990B909310018093D5
:104610000F0114C0913029F49093AD038091AC0345
:10462000F1CF923009F09AC020910D0130910E0126
:1046300030930C0320930B039093AD038091AD0353
:10464000813009F0C3C08091FD029FEF980F923036
:1046500008F0FDC0813009F049C0EE24E394F12C4C
:1046600000E110E020E430E040E65CE070E060E073
:1046700090E080E00E94061220E430E040EE59E035
:1046800060E170E090E080E00E94061280912001DD
:104690000E94AC1A8130F9F41092AB031092AA0375
:1046A00010929A0310929B0310929C0310929D0308
:1046B0001092960310929703109298031092990308
:1046C00010929E0310929F031092A0031092A103D8
:1046D00082E08093FD0280911F010E94AC1A81301C
:1046E00029F41092FD0287E08093AD038091FD02D2
:1046F000823019F5EE24E394F12C00E110E020E47F
:1047000030E040EE5CE070E060E090E080E00E942D
:10471000061220E130E044E150E061E070E08EE517
:1047200092E00E94891C83E00E94AC1A813029F437
:104730001092FD0287E08093AD03DF91CF911F912E
:104740000F91FF90EF90DF90CF90BF90AF909F9030
:104750008F907F906F905F904F900895933051F4B9
:1047600080910B0190910C0190930C0380930B03AB
:1047700082E003C0943021F481E08093AD035ECFEA
:10478000953071F480911401882329F080910901FA
:1047900090910A01E9CF8091070190910801E4CF3F
:1047A000963051F3973031F481E08093AD038091DE
:1047B000A40328CF983031F481E08093AD03809139
:1047C000140120CF9930C1F28091AD03C091B303A1
:1047D000823009F0FFC48091FF02909100030091A4
:1047E0000B0310910C03863091050CF496C31092C4
:1047F00000031092FF0281E08093FE020C591F4FCC
:1048000010930C0300930B03A3C38330E9F681E0FC
:104810008093AD0381E090E090930A0380930903B5
:104820002BE030E030930601209305011092050340
:1048300010920603109207031092080310920103CE
:10484000109202031092030310920403DECEC09173
:10485000B30380912001C111C3C00E94AC1A009122
:104860000F0110911001813019F5015011091093B9
:10487000100100930F0180910F019091100183307E
:1048800091050CF452C082E090E090931001809367
:104890000F0180910F01909110018130910509F471
:1048A0004BC0C0E0D0E0029709F048C0C1E045C06D
:1048B00080911F010E94AC1A813019F40F5F1F4FC5
:1048C000D6CF83E00E94AC1A8130A9F697E090938E
:1048D000AD030115110591F41092940380E090E06E
:1048E000A0E0BFE38093010190930201A093030134
:1048F000B093040185E080930001BDCF0130110524
:1049000019F480939403EACF82E08093940380E0CB
:1049100090E0A0EAB0E48093010190930201A0939B
:104920000301B093040183E0E6CF97FFB2CF10926A
:10493000100110920F01ADCFC0E0D1E0CC2ED12CF0
:10494000760101E010E020E430E048E156E070E05C
:1049500060E090E080E00E94061220E430E048E150
:1049600056E061E070E090E080E00E94061220E7EF
:10497000D29F50011124A50148595F4F0EE010E06D
:1049800020E430E062E070E090E080E00E940612F7
:1049900081E0C827D0E07E0101E010E020E430E0B3
:1049A00048E156E060E170E090E080E00E9406128D
:1049B00020E430E048E156E061E170E090E080E022
:1049C0000E940612A50148525F4F0EE010E020E45D
:1049D00030E062E170E090E080E00E940612ADCE2F
:1049E00092E09093320410922B0410922A041092B9
:1049F0002D0410922C040E94AC1A813031F481E015
:104A000090E09093100180930F0180911F010E940C
:104A1000AC1A813021F41092100110920F01809194
:104A2000090390910A03181619060CF05EC1209133
:104A30000F01309110012130310571F060E084E602
:104A400090E00E948032109221018FEF9FEF9093AF
:104A50000A03809309036ECE1092A5031092A2035D
:104A600081309105A9F5909331048093300490939F
:104A70002F0480932E0410922B0410922A0410927B
:104A80002D0410922C0483E692E00E94171C1092D1
:104A90002B0410922A0480E190E090932D048093DF
:104AA0002C0488E792E00E94171C83E00E94AC1A55
:104AB000813009F042CE8BE090E090930601809324
:104AC000050182E090E090930A038093090335CEBC
:104AD0008230910509F04AC03093310420933004AC
:104AE00030932F0420932E0410922B0410922A044A
:104AF00010922D0410922C048091050190910601D2
:104B0000009771F589E692E00E94171C10922B0421
:104B100010922A0480E190E090932D0480932C045D
:104B20008091050190910601892BE9F48FE692E0CE
:104B30000E94171C83E00E94AC1A813009F0FDCD61
:104B40008091050190910601892B09F0F6CD8BE04B
:104B500090E0909306018093050183E090E0B3CF4D
:104B60000E94BB1CD3CF87E792E0E2CF039709F006
:104B7000E4CD309331042093300430932F042093FC
:104B80002E0410922B0410922A0410922D041092DD
:104B90002C0489E692E00E94171C10922B041092BC
:104BA0002A0480E190E090932D0480932C0480915E
:104BB000050190910601009709F08AC089E692E00C
:104BC0000E94171C83E00E94AC1A813009F0B5CD19
:104BD0008091050190910601892B09F0AECD80905E
:104BE000010390900203A0900303B0900403C090CF
:104BF0000503D0900603E0900703F0900803C092ED
:104C00008403D0928503E0928603F092870380921A
:104C1000800390928103A0928203B09283038C144C
:104C20009D04AE04BF0469F4D501C4010196A11D21
:104C3000B11D8093840390938503A0938603B09362
:104C4000870307E010E05AE0452E512C612C712CAF
:104C5000C02FC701B601A30192010E94E0340531C3
:104C6000D1F1C8010E948032C33151F0C701B601B1
:104C7000A30192010E94E03469017A01C53169F112
:104C8000C501B401A30192010E94E034C80101965C
:104C90000E948032C33141F0C501B401A3019201E9
:104CA0000E94E03449015A010E5F1F4F0731110580
:104CB00079F60E94771B61E084E690E00E948032E2
:104CC00081E08093210110920A031092090332CDF2
:104CD0000E94BB1C77CF622FC4CFC501B401A301D2
:104CE00092010E94E034622FD1CFC83009F042C057
:104CF00080910F0190911001019751F5F12CE12C59
:104D000000E110E020E430E040EE5AE070E060E0C6
:104D100090E080E00E940612EE24E394F12C20E45F
:104D200030E040E65AE060E170E090E080E00E9410
:104D3000061283E00E94AC1A813009F0FECC60912B
:104D40000F01609314018EE190E00E948032F2CC5A
:104D5000EE24E394F12C00E110E020E430E040EE9A
:104D60005AE070E060E090E080E00E940612F12CD2
:104D7000E12CD5CFC93019F581E090E09093310452
:104D80008093300490932F0480932E048EE792E05A
:104D90000E94171C10922B0410922A0480E190E0CC
:104DA00090932D0480932C0484E892E00E94171CB9
:104DB00083E00E94AC1A813009F0BFCCBBCC80915B
:104DC0000F01909110018130910509F05CC0EE2433
:104DD000E394F12C00E110E020E430E0C43071F500
:104DE00040EE5DE060E170E090E080E00E9406123D
:104DF000F12CE12C20E430E040E65DE070E060E082
:104E000090E080E00E94061283E00E94AC1A81309C
:104E100009F093CC20910F01309110012130310520
:104E200009F08BCC9091B3039130B9F41092FD024C
:104E300087E08093AD039093AC037FCC40EE5BE0C2
:104E400060E170E090E080E00E940612F12CE12C1D
:104E500020E430E040E65BE0D1CF943039F490912B
:104E6000FD0291116ACC8093FD0267CC963019F453
:104E70008093B8035FCC973009F05FCC9093AD037B
:104E80008093A4035ACC892B09F057CCF12CE12C48
:104E900000E110E020E430E0C43021F540EE5DE0B8
:104EA00060E170E090E080E00E940612EE24E3945E
:104EB000F12C20E430E040E65DE070E060E090E05E
:104EC00080E00E94061283E00E94AC1A813009F053
:104ED00034CC8091B3038130A9F41092FD0210927A
:104EE000AC0328CC40EE5BE060E170E090E080E055
:104EF0000E940612EE24E394F12C20E430E040E618
:104F00005BE0DBCF863019F41092B80313CC873006
:104F100009F010CC1092A4030DCC8B3F9F4F54F49A
:104F2000109200031092FF0281E08093FE0204566B
:104F3000110966CC80911F010E94AC1A813009F0E2
:104F400061C08091FE02882309F459C01092FE02CC
:104F500000910B0310910C03C23009F061C00D33B6
:104F6000110534F08CE390E090930C0380930B03D5
:104F700083E00E94AC1A813059F480910B03909128
:104F80000C0390930E0180930D0187E08093AD0395
:104F900030E020E048E250E063E070E08AE892E030
:104FA0000E94891C80910B0390910C03029734F4AA
:104FB00082E090E090930C0380930B0320910B030D
:104FC00030910C038091B303853009F4BBC050E0ED
:104FD00040E070E060E083E090E0DF91CF911F91CE
:104FE0000F91FF90EF90DF90CF90BF90AF909F9088
:104FF0008F907F906F905F904F900C949D1C0F5FEF
:105000001F4FFECB809120010E94AC1A813009F025
:105010009FCF8091FE02811199CF01501109F0CBF1
:10502000C33011F50531110534F084E190E090931F
:105030000C0380930B0383E00E94AC1A813059F477
:1050400080910B0390910C0390930C0180930B01C2
:1050500087E08093AD0330E020E048E250E063E079
:1050600070E08CE892E09CCFC53009F09BCF809136
:1050700020010E946F0D892BC9F51092A503109293
:10508000A2038091FF02909100038B3F2FEF9207C4
:1050900054F10197909300038093FF0283E00E94F4
:1050A000AC1A813009F07ECFB801012E000C880BBC
:1050B000990B0E94AA3320911401222391F110939D
:1050C0000A010093090120E030E048E651E40E9423
:1050D0005F340E947233709308016093070187E088
:1050E0008093AD035FCF8AEF9FEFD4CF80911F01F4
:1050F0000E946F0D892B81F41092A5031092A203D8
:105100008091FF02909100038630910514F401967E
:10511000C1CF86E090E0BECF109200031092FF0254
:10512000BDCF20E030E048E651E40E9400330E9409
:10513000723370930A016093090110930801009380
:105140000701CDCF80911401882319F1283E334007
:1051500034F087EE93E090930C0380930B036091FF
:105160000B0370910C03072E000C880B990B0E9407
:10517000AA330E94BD18EE24E394F12C00E210E063
:1051800020E130E040EE50E170E060E080E390E04C
:1051900024CC2031374234F08FE097E290930C0317
:1051A00080930B0360910B0370910C03072E000C8E
:1051B000880B990B0E94AA330E94BD18EE24E39439
:1051C000F12C00E110E020E130E040E252E160E14A
:1051D00070E0DCCFC2300CF457C0C4300CF45AC0BD
:1051E000C6300CF45EC0C8300CF462C0CA300CF497
:1051F00066C02C2F2170522ED0E7C814D9040CF0B1
:1052000065C0560181E0A822BB249A2D8B2DA114E4
:10521000B10419F020E1A22EB12C692E782E552070
:1052200031F036016094709421E06222772473019A
:1052300001E010E020E430E048E156E0B50190E004
:1052400080E00E940612B5016F5F7F4F20E430E0DE
:1052500048E156E090E080E00E940612DC9DA0014B
:10526000DD9D500D112448545E4FB5016E5F7F4F98
:105270000EE010E020E430E090E080E00E940612B2
:105280008FEFC81AD80AB9CFB2E08B2E912CD12C4F
:10529000C12CAFCFF4E08F2E912CA2E0CA2ED12CDE
:1052A000A8CF76E0872E912CE4E0CE2ED12CA1CF92
:1052B00058E0852E912C66E0C62ED12C9ACF3AE08C
:1052C000832E912C48E0C42ED12C93CF1092AD03A5
:1052D000C930ECF480911F010E94AC1A813019F49E
:1052E000CF5FC093B303C091B3031C16F4F4809155
:1052F00020010E94AC1A813019F4C150C093B3034D
:105300008091B3038A30F1F41092AE0316CAC9300B
:1053100051F780911F010E94AC1AC091B3038230F3
:1053200031F78AE08093B303DECFC111E9CF8091DA
:1053300020010E94AC1A823009F0FFC98FEF8093E0
:10534000B303DECF8F3F09F0F8C983E08093AE034B
:10535000F4C91F920F920FB60F9211242F933F930F
:105360008F939F93AF93BF9380917803909179032C
:10537000A0917A03B0917B033091770326E0230F4D
:105380002D3758F50296A11DB11D20937703809308
:10539000780390937903A0937A03B0937B03809171
:1053A0007C0390917D03A0917E03B0917F030196D1
:1053B000A11DB11D80937C0390937D03A0937E0378
:1053C000B0937F03BF91AF919F918F913F912F91A8
:1053D0000F900FBE0F901F90189529E8230F03968A
:1053E000A11DB11DD2CF1F920F920FB60F921124A3
:1053F0002F933F934F935F936F937F938F939F93DD
:10540000AF93BF93EF93FF93E0911B01F0911C01C9
:105410000995FF91EF91BF91AF919F918F917F91EE
:105420006F915F914F913F912F910F900FBE0F9011
:105430001F9018951F920F920FB60F9211242F9361
:105440003F934F935F936F937F938F939F93AF930C
:10545000BF93EF93FF93E0911901F0911A01099521
:10546000FF91EF91BF91AF919F918F917F916F913C
:105470005F914F913F912F910F900FBE0F901F9012
:1054800018951F920F920FB60F9211248F930FB69B
:10549000F894A895809160008861809360001092D4
:1054A00060000FBE8F910F900FBE0F901F90189548
:1054B0001F920F920FB60F9211242F933F934F9389
:1054C0005F936F937F938F939F93AF93BF93EF936C
:1054D000FF938091B900887F803609F44AC0F0F5C7
:1054E000883209F4A7C018F5803109F49BC0B8F4DC
:1054F000882309F4F9C0883009F494C0FF91EF9132
:10550000BF91AF919F918F917F916F915F914F91DB
:105510003F912F910F900FBE0F901F9018958831DB
:1055200009F488C0803251F78093E30314C08034BB
:1055300009F49DC040F48033B9F38833F9F68093C1
:10554000E30385ECB0C0803509F485C0883509F4E3
:1055500096C0883499F60E945815D0CF883909F43E
:105560008CC038F5883729F050F4883611F0803730
:1055700029F683E08093E5031092760357C08838BC
:1055800009F47BC0803919F0803809F0B7CF8091D9
:105590007603803208F071C0E091760381E08E0FCF
:1055A000809376038091BB00F0E0EA5AFC4F808341
:1055B0003DC0803B39F0E0F4803A09F479C0883A84
:1055C00009F09CCF84E08093E5031092550310927C
:1055D0005403E0918A03F0918B0309958091540361
:1055E00081110FC081E0809354031092340309C0ED
:1055F000803C09F4A6CF883C09F4A3CF883B09F08E
:105600007DCFE091550381E08E0F80935503F0E04C
:10561000EC5CFC4F80818093BB009091550380919E
:10562000540329C08091C0038093BB0085EC809314
:10563000BC0064CF9091E2038091E103981758F584
:10564000E091E20381E08E0F8093E203F0E0EF53FC
:10565000FC4F8081E9CFE091E20381E08E0F8093DF
:10566000E2038091BB00F0E0EF53FC4F8083909108
:10567000E2038091E1039817C8F285E8D8CFE09162
:10568000E20381E08E0F8093E2038091BB00F0E0A3
:10569000EF53FC4F80838091E40381115CCF81E064
:1056A0008093BF0384EA8093BC001092E50326CF69
:1056B00085EC8093BC001092E503809176038032E4
:1056C00030F4E0917603F0E0EA5AFC4F10826091EA
:1056D000760370E0E0918803F091890386E593E01A
:1056E0000995109276030ACF1092E30334CF1F92EC
:1056F0000F920FB60F9211242F933F934F935F9306
:105700006F937F938F939F93AF93BF93EF93FF9389
:1057100080910A0490910B048093B2008091100351
:1057200090911103A0911203B09113030196A11D52
:10573000B11D8093100390931103A0931203B093B3
:1057400013038091100390911103A0911203B09163
:10575000130340910E0450910F0460911004709156
:10576000110484179507A607B70710F180910F035E
:1057700081111EC081E080930F03809110039091EE
:105780001103A0911203B0911303841B950BA60B78
:10579000B70B8093100390931103A0931203B0935F
:1057A0001303E0910C04F0910D04099510920F037E
:1057B000FF91EF91BF91AF919F918F917F916F91E9
:1057C0005F914F913F912F910F900FBE0F901F90BF
:1057D0001895E2E1F4E01382128288EE93E0A0E0F3
:1057E000B0E084839583A683B78387E392E09183B7
:1057F0008083EEE1F4E01382128220E430E035830E
:10580000248380E290E09783868331872087938783
:105810008287158A158614861786168681E0848B02
:105820002FEF3FEF338B228B318B208B868B87E4DE
:1058300092E0918380838FEF818F858F838F828F1A
:1058400084E0848F0895789484B5826084BD84B5A3
:10585000816084BD85B5826085BD85B5816085BD6B
:1058600080916E00816080936E0010928100809123
:1058700081008260809381008091810081608093AB
:105880008100809180008160809380008091B100D0
:1058900084608093B1008091B00081608093B000FB
:1058A00080917A00846080937A0080917A0082608F
:1058B00080937A0080917A008E7F80937A00809125
:1058C0007A00806880937A001092C10083E0809310
:1058D0001301C0911F0160E0809120010E94C60D5C
:1058E00060E083E00E94C60D60E08C2F0E94C60D30
:1058F00062E082E00E94C60D61E08DE00E94C60D6C
:10590000C7E0D0E0CE010E9478324090150150905F
:1059100016016090170170901801A82FB0E0A30144
:1059200092010E9402350091840310918503209119
:105930008603309187036B017C01C00ED11EE21EED
:10594000F31EC0928403D0928503E0928603F09206
:105950008703CE0101960E947832A82FB0E0A30100
:1059600092010E94023500918003109181032091E1
:105970008203309183034B015C01800E911EA21EB5
:10598000B31E8092800390928103A0928203B09212
:105990008303AAE0B0E092010E94023560931501F2
:1059A0007093160180931701909318012296C731C6
:1059B000D10509F0A7CFC814D904EA04FB0469F49F
:1059C0008FEFC81AD80AE80AF80AC0928403D09266
:1059D0008503E0928603F09287030E94771B84E69A
:1059E00090E00E947832809321018EE190E00E9445
:1059F0007832809314010E94E81BC2E0C093360401
:105A00008CE380933504809137048F3F09F4D2C131
:105A100061E0809139040E94C60D61E080913B04F1
:105A20000E94C60D80913B04082E000C990BFC01CE
:105A3000E957F84EE491F0E0EE0FFF1FE358F84EFF
:105A4000259134913093420420934104FC01EA599A
:105A5000F84EE491E093470480913904082E000C3D
:105A6000990BFC01E957F84EE491F0E0EE0FFF1FAF
:105A7000E358F84E25913491309344042093430425
:105A8000FC01EA59F84EE491E093480480913C040B
:105A900081113EC061E0809137040E94C60D61E033
:105AA000809138040E94C60D80913804082E000CA5
:105AB000990BFC01E957F84EE491F0E0EE0FFF1F5F
:105AC000E358F84E259134913093400420933F04DD
:105AD000FC01EA59F84EE491E093460480913704C2
:105AE000082E000C990BFC01E957F84EE491F0E008
:105AF000EE0FFF1FE358F84E2591349130933E048A
:105B000020933D04FC01EA59F84EE491E0934504EA
:105B100080913C04882309F437C0CFB7F894809172
:105B20008E03811127C0E1E9F7E18491E0E7F7E115
:105B30009491E82FF0E0EE0FFF1FE45AF84EA59184
:105B4000B491EC91E92321F461E08AE00E94980D80
:105B500061E08AE00E94C60D8CB580618CBD8CB579
:105B600080648CBD61E08DE00E94C60D61E08BE039
:105B70000E94C60D80918E038F5F80938E03CFBFEE
:105B800080E58CBD81E08DBD80913A0487FD1EC00B
:105B900061E00E94C60D61E080913A040E94980D78
:105BA00061E070E080E090E00E94270E60E080916C
:105BB0003A040E94980D6AE070E080E090E00E9454
:105BC000270E61E080913A040E94980D8EEA0E94AF
:105BD0000F1685ED0E940F1680E80E940F1688EAC6
:105BE0000E940F168FE10E940F1683ED0E940F1680
:105BF00080E00E940F1680E40E940F168DE80E943C
:105C00000F1684E10E940F1680E20E940F1680E0BA
:105C10000E940F1681EA0E940F1688EC0E940F1650
:105C20008AED0E940F1682E10E940F1681E80E9401
:105C30000F168FEC0E940F1689ED0E940F1681EF50
:105C40000E940F1689ED0E940F1681EF0E940F1619
:105C50008BED0E940F1680E40E940F1684EA0E94CA
:105C60000F1686EA0E940F168EE20E940F168FEA28
:105C70000E940F160E94510C0E94F81662E080E00C
:105C80000E94C60D83E19DE090931A018093190153
:105C9000809169008C7F826080936900E89A86EF2A
:105CA0009BE190931C0180931B0180916900837F8D
:105CB000886080936900E99A60E0A62E60E0B62EC5
:105CC00099249A94CC24C394D12CD3E0C2E0E9E087
:105CD0006E2EF5E08F2E44E0542E56E0752E109176
:105CE000BC038FEF810F823008F0B5C082E00E94C4
:105CF0006F0D892B09F094C0113021F40E946316B6
:105D0000C093BC038091BC03823009F04CC00E9458
:105D1000262281E80E940F1680E00E940F168091D3
:105D20008F03823314F010928F0380918F038F5F63
:105D300080938F03EE24E394F12C0FE010E02DE12B
:105D400030E042E050E062E170E08EE194E00E94D9
:105D5000391480918F03181624F467E184E10E94BE
:105D6000351580918F038B3024F06DE189E10E941D
:105D7000351580918F03853124F062E28FE10E9416
:105D8000351580918F038F3124F067E284E20E9401
:105D9000351580918F03893224F06CE289E20E94EC
:105DA00035150E946B16A114B10409F498CF0E9416
:105DB000000091CF10928D0310928C031092E70394
:105DC000109209041092E50381E08093E40310929D
:105DD000BF0361E082E10E94980D61E083E10E94CF
:105DE000980D8091B9008E7F8093B9008091B900A1
:105DF0008D7F8093B90080E28093B80085E4809322
:105E0000BC0087E19DE090938B0380938A0388E137
:105E10009DE09093890380938803C093B800B4CE2B
:105E20001092BC030E94510C0E94F816109292032B
:105E300081E080932201C09391031092A5031092F8
:105E40009003109295039091A403933009F0ABCF87
:105E50008093A403A8CF8091220118160CF009C3E7
:105E6000843029F4C09322010E9463169CCF8230B3
:105E700009F099CF8091B803813039F48091B7034C
:105E80008F5F8093B7031092B8030E94262210916F
:105E9000B50381E80E940F16812F0E940F164091D2
:105EA000B70320912204309123048091240490911F
:105EB000250440FD93C08092200170921F01C09381
:105EC000330430932704209326049093290480936D
:105ED00028048091B403882331F09091B30391504A
:105EE000983008F482C0D092B203C092B10390916E
:105EF000B0038F3F29F02FEF290F233008F0D1C0D6
:105F0000913009F061C0EE24E394F12C01E010E03F
:105F10002EE330E041E050E065E070E08EE194E097
:105F20000E9488140EE110E02EE330E04EE150E0D4
:105F300065E070E08EE194E00E94881408E010E0D3
:105F400024E030E048E050E061E070E08EE194E071
:105F50000E94881408E110E024E030E048E150E0BD
:105F600061E070E08EE194E00E94881421E030E06E
:105F700048E050E061E070E08EE194E00E94881417
:105F80000EE110E025E030E041E050E065E070E037
:105F90008EE194E00E9488142EE330E041E050E06E
:105FA0006EE370E08EE194E00E9488149091930378
:105FB00081E0890F8093930390FD1CC064E670E03C
:105FC00080E090E00E94270E8091B003823009F0BB
:105FD000E8CED093B00310922201E3CE709220015C
:105FE00080921F01109233046CCF1092B203109272
:105FF000B1037DCFEE24E394F12C05E110E02DE117
:1060000030E049E050E061E170E08EE194E00E9410
:10601000881404E110E02DE130E049E050E062E155
:1060200070E08EE194E00E94881406E110E02EE119
:1060300030E049E050E06EE170E08EE194E00E94D3
:10604000881407E110E02FE130E04AE050E06FE112
:1060500070E08EE194E00E9488142CE230E04BE086
:1060600050E060E270E08EE194E00E9488142BE240
:1060700030E04CE050E060E270E08EE194E00E949D
:10608000881464E670E080E090E00E94270E809122
:106090009303843109F098CFC093B0031092930317
:1060A00093CF811142C080911D0190911E018C30CF
:1060B0009105ACF0019790931E0180931D01EE2491
:1060C000E394F12C06E110E020E430E04EE957E1E2
:1060D00065E070E082E090E00E94061262CE8B30B4
:1060E000910581F462E370E080E090E00E94270E69
:1060F0008AE090E090931E0180931D0181E08093DF
:10610000AF034FCE0A9709F04CCE9092B30381E0D3
:106110008093B4031092AE031092AD0384E190E03B
:1061200090931E0180931D013CCE0091AC038EEF35
:10613000800F8230E0F4023021F40E946316D09385
:10614000AC034091AA035091AB036091A6037091F8
:10615000A7038091A8039091A9030E943122809106
:10616000A503823009F01DCE5092AC031ACE1091D7
:10617000A403812F8D7F813021F48091A30381308E
:10618000F1F1123009F079C08091A403813051F40B
:10619000C093A4031092AE031092A5031092A20321
:1061A0000E9463168091AE0381112EC04091AA0314
:1061B0005091AB036091A6037091A7038091A8034F
:1061C0009091A9030E94312280911F010E94AC1A74
:1061D000F090AE03813009F041C0F394F092AE0329
:1061E0008091AE03843009F042C01092AE038091DA
:1061F000A503823009F0D5CDD093A403D2CD1330BE
:1062000019F68093A403C0CF813071F460919E038E
:1062100070919F038091A0039091A1030E9472331B
:10622000CB010E94EE19D0CF823059F460919A03CD
:1062300070919B0380919C0390919D030E949918FB
:10624000C3CF833009F660919603709197038091D4
:106250009803909199030E947518B6CF8091200100
:106260000E94AC1A813009F0BBCFFA94B7CF8F3FB0
:1062700009F0BDCFD093AE03BACF8091A5039EEFB6
:10628000980F9230E8F5833031F50E94AC1AF82E61
:1062900081E0F81220C00E9463161092A5031092AC
:1062A000A203133051F4F092A4031092B4038BE0D4
:1062B00090E090931E0180931D01043009F071CD90
:1062C00081E08093AC031092B4038BE090E0909354
:1062D0001E0180931D018091A503823009F061CDDC
:1062E0008EEA0E940F161092BA031092B903D09250
:1062F000BE03C092BD03D093A5031092950351CD68
:1063000080919403982F9D7F49F58091B3038A3043
:1063100011F08F3F01F580911F010E94AC1A82306D
:1063200089F41092B3034091AA035091AB0360919A
:10633000A6037091A7038091A8039091A9030E94DE
:1063400031222FCD809120010E94AC1A823059F762
:106350006092B303E8CF0E94E02223CD813009F0A0
:1063600020CD8091B3038A3011F08F3FA1F7809147
:10637000AE03811132C04091AA035091AB036091EA
:10638000A6037091A7038091A8039091A9030E948E
:1063900031221091AE0313300CF04AC080911F01DE
:1063A0000E94AC1A813019F41F5F1093AE03F09075
:1063B000AE031F140CF04BC0809120010E94AC1A58
:1063C000813019F4FA94F092AE038091AE038530D7
:1063D00009F049C01092B303E4CC813071F46091AC
:1063E0009E0370919F038091A0039091A1030E944E
:1063F0007233CB010E94EE19CCCF823059F46091F8
:106400009A0370919B0380919C0390919D030E943D
:106410009918BFCF833009F0BCCF6091960370917B
:10642000970380919803909199030E947518B1CFBA
:10643000133009F0BCCF80911F010E94AC1AF0907C
:10644000AE03823009F0B8CF8092AE03B0CFF11026
:10645000BCCF809120010E94AC1A823009F0A1CCFF
:106460009092AE03B2CF8F3F09F09BCC6092B30302
:1064700098CC811118C00E94262281E80E940F1634
:1064800080E00E940F160E946B16909222018EEA05
:106490000E940F161092BA031092B903D092BE0355
:1064A000C092BD0380CC8F3F09F07DCC809121014B
:1064B000863019F481E08093210161E08FE00E9431
:1064C000980D61E082E10E94980D61E083E10E94F5
:1064D000980D60E08DE00E94980D30E020E050E0E3
:1064E00040E06AE070E08BEB93E00E945A0E5BCCD8
:1064F000F999FECF92BD81BDF89A992780B508958C
:10650000262FF999FECF1FBA92BD81BD20BD0FB6CF
:10651000F894FA9AF99A0FBE019608955058BB273D
:10652000AA270E94A6320C9420340E94123438F01C
:106530000E94193420F039F49F3F19F426F40C948A
:106540000F340EF4E095E7FB0C940934E92F0E9418
:10655000313458F3BA17620773078407950720F0A0
:1065600079F4A6F50C9453340EF4E0950B2EBA2F63
:10657000A02D0B01B90190010C01CA01A001112449
:10658000FF27591B99F0593F50F4503E68F11A16F5
:10659000F040A22F232F342F4427585FF3CF469586
:1065A00037952795A795F0405395C9F77EF41F16A8
:1065B000BA0B620B730B840BBAF09150A1F0FF0F72
:1065C000BB1F661F771F881FC2F70EC0BA0F621F5E
:1065D000731F841F48F4879577956795B795F7954E
:1065E0009E3F08F0B0CF9395880F08F09927EE0FE3
:1065F0009795879508950E94E53308F481E0089502
:106600000E9414330C9420340E94193458F00E94D4
:10661000123440F029F45F3F29F00C9409345111F1
:106620000C9454340C940F340E94313468F3992341
:10663000B1F3552391F3951B550BBB27AA2762177E
:106640007307840738F09F5F5F4F220F331F441F8B
:10665000AA1FA9F335D00E2E3AF0E0E832D09150BF
:106660005040E695001CCAF72BD0FE2F29D0660FAC
:10667000771F881FBB1F261737074807AB07B0E8EF
:1066800009F0BB0B802DBF01FF2793585F4F3AF0F5
:106690009E3F510578F00C9409340C9454345F3FBC
:1066A000E4F3983ED4F3869577956795B795F7957B
:1066B0009F5FC9F7880F911D9695879597F9089563
:1066C000E1E0660F771F881FBB1F621773078407FF
:1066D000BA0720F0621B730B840BBA0BEE1F88F70E
:1066E000E09508950E9479336894B1110C94543464
:1066F00008950E94393488F09F5798F0B92F992750
:10670000B751B0F0E1F0660F771F881F991F1AF09C
:10671000BA95C9F714C0B13091F00E945334B1E07A
:1067200008950C945334672F782F8827B85F39F079
:10673000B93FCCF3869577956795B395D9F73EF435
:1067400090958095709561957F4F8F4F9F4F0895DD
:10675000E89409C097FB3EF49095809570956195FB
:106760007F4F8F4F9F4F9923A9F0F92F96E9BB27B1
:106770009395F695879577956795B795F111F8CF2D
:10678000FAF4BB0F11F460FF1BC06F5F7F4F8F4F98
:106790009F4F16C0882311F096E911C0772321F08E
:1067A0009EE8872F762F05C0662371F096E8862F26
:1067B00070E060E02AF09A95660F771F881FDAF77D
:1067C000880F9695879597F90895990F0008550FAA
:1067D000AA0BE0E8FEEF16161706E807F907C0F067
:1067E00012161306E407F50798F0621B730B840B6F
:1067F000950B39F40A2661F0232B242B252B21F449
:1068000008950A2609F4A140A6958FEF811D811DE8
:10681000089597F99F6780E870E060E008959FEF22
:1068200080EC089500240A94161617061806090627
:10683000089500240A9412161306140605060895F6
:10684000092E0394000C11F4882352F0BB0F40F47E
:10685000BF2B11F460FF04C06F5F7F4F8F4F9F4FBE
:10686000089557FD9058440F551F59F05F3F71F040
:106870004795880F97FB991F61F09F3F79F08795A7
:106880000895121613061406551FF2CF4695F1DF30
:1068900008C0161617061806991FF1CF86957105C0
:1068A000610508940895E894BB2766277727CB01F4
:1068B00097F908950E94E53308F48FEF08950E9438
:1068C00072340C9420340E94123438F00E9419342F
:1068D00020F0952311F00C9409340C940F341124FA
:1068E0000C9454340E94313470F3959FC1F3950F8A
:1068F00050E0551F629FF001729FBB27F00DB11D44
:10690000639FAA27F00DB11DAA1F649F6627B00DD3
:10691000A11D661F829F2227B00DA11D621F739FBC
:10692000B00DA11D621F839FA00D611D221F749FCA
:106930003327A00D611D231F849F600D211D822F11
:10694000762F6A2F11249F5750409AF0F1F0882338
:106950004AF0EE0FFF1FBB1F661F771F881F915065
:106960005040A9F79E3F510580F00C9409340C94D7
:1069700054345F3FE4F3983ED4F38695779567955A
:10698000B795F795E7959F5FC1F7FE2B880F911D8F
:106990009695879597F9089597FB072E16F400941E
:1069A00007D077FD09D00E940D3507FC05D03EF4D5
:1069B000909581959F4F0895709561957F4F0895AB
:1069C000A1E21A2EAA1BBB1BFD010DC0AA1FBB1FF3
:1069D000EE1FFF1FA217B307E407F50720F0A21B65
:1069E000B30BE40BF50B661F771F881F991F1A94D2
:1069F00069F760957095809590959B01AC01BD01FC
:106A0000CF0108950E942735A59F900DB49F900D4A
:106A1000A49F800D911D11240895AA1BBB1B51E159
:106A200007C0AA1FBB1FA617B70710F0A61BB70BFE
:106A3000881F991F5A95A9F780959095BC01CD01A3
:106A40000895EE0FFF1F0590F491E02D0994A29F89
:106A5000B001B39FC001A39F700D811D1124911D32
:106A6000B29F700D811D1124911D089581E090E069
:0A6A7000F8940C943B35F894FFCF26
:106A7A00050000003F0B00AA0564000F000A000190
:106A8A00001A1E010101000000590E000014000640
:106A9A0005010100000000000000000000000000E5
:106AAA0000000000000000000000000000000000DC
:106ABA0000000000000000000000000000000000CC
:106ACA0000000000000000000000000000000000BC
:106ADA00000080808000000000000000000000002C
:106AEA00000000008080C0C000000000000000001C
:106AFA00000000000000000000000000000000008C
:106B0A00000000000000000000000000000000007B
:106B1A00000000000000000000000000000000006B
:106B2A000000000000000080C0E0F0F8FCF8E0007F
:106B3A00000000000000000000000000000000004B
:106B4A0080808080800080800000000080808080BB
:106B5A008000FFFFFF00000000808080800000802E
:106B6A0080000080FFFF808000808000808080801D
:106B7A000080800000000000808000008C8E84006D
:106B8A000080F8F8F8800000000000000000000013
:106B9A00000000000103070F1F3F7F0080C0E0F0E4
:106BAA00F8FCFE00000000E015B315AC1599158A33
:106BBA00158915000000008512190D62118814A8A4
:106BCA000E05103914D713BA1384120D0A0065780A
:106BDA006974003E3330304200446F6E65210020F4
:106BEA003E3530424152002035304241520056353E
:0E6BFA002E3030003231443138006D0073000F
:107E000001C0ABC0112484B7882361F0982F9A7009
:107E1000923041F081FF02C097EF94BF282E80E09E
:107E2000BFD0EEC085E08093810082E08093C000E7
:107E300088E18093C10089E18093C40086E080934B
:107E4000C2008EE0ADD0259A84E028E13EEF91E0BB
:107E5000309385002093840096BBB09BFECF1D9A83
:107E6000A8954091C00047FD02C0815089F78CD091
:107E7000813461F489D0182F99D01238E9F0113883
:107E800011F488E001C083E078D064C0823411F43A
:107E900084E103C0853419F485E090D05BC085355A
:107EA00039F472D0C82F70D0D82FCC0FDD1F51C03D
:107EB000863521F484E082D080E0E6CF843661F517
:107EC00063D062D0D82E60D0F82E00E011E05CD0F4
:107ED000F80181938F01DE12FACF68D0F5E4FF122A
:107EE00001C0FFCF40E050E063E0CE0136D07E011C
:107EF00000E011E0F801419151918F0161E0C7016B
:107F00002CD0F2E0EF0EF11CD012F4CF40E050E0A4
:107F100065E0CE0122D01EC0843771F435D034D054
:107F2000F82E32D043D08E01F80185918F0125D0F3
:107F3000FA94F110F9CF0EC0853739F437D08EE1BD
:107F40001CD085E91AD08FE09FCF813511F488E0ED
:107F500027D02CD080E111D08ACFFC010A0167BF65
:107F6000E895112407B600FCFDCF667029F0452B7B
:107F700019F481E187BFE89508959091C00095FFBD
:107F8000FCCF8093C60008958091C00087FFFCCF8E
:107F90008091C00084FD01C0A8958091C60008951D
:107FA000E0E6F0E098E1908380830895EDDF803291
:107FB00019F088E0F5DFFFCF84E1DFCFCF93C82F42
:0A7FC000E3DFC150E9F7CF91F1CFE4
:027FFE00000879
:0400000300007E007B
:00000001FF
